S02700002E2E5C62696E5C6F70656E626C745F6F6C696D65785F73746D3332703430352E73726563AE
S3150800000000000220A12E0008EF2E0008F12E00089D
S31508000010F32E0008F52E0008F72E00080000000051
S31508000020000000000000000000000000F92E000893
S31508000030FB2E000800000000FD2E0008FF2E000819
S31508000040032F0008052F0008072F0008092F0008AE
S315080000500B2F00080D2F00080F2F0008112F00087E
S31508000060132F0008152F0008172F0008192F00084E
S315080000701B2F00081D2F00081F2F0008212F00081E
S31508000080232F0008252F0008272F0008292F0008EE
S315080000902B2F00082D2F00082F2F0008312F0008BE
S315080000A0332F0008352F0008372F0008392F00088E
S315080000B03B2F00083D2F00083F2F0008412F00085E
S315080000C0432F0008452F0008472F0008492F00082E
S315080000D04B2F00084D2F00084F2F0008512F0008FE
S315080000E0532F0008552F0008572F0008592F0008CE
S315080000F05B2F00085D2F00085F2F0008612F00089E
S31508000100632F0008652F0008672F0008692F00086D
S315080001106B2F00086D2F00086F2F0008712F00083D
S31508000120732F0008752F0008772F0008792F00080D
S315080001307B2F00087D2F00087F2F0008812F0008DD
S31508000140832F0008852F0008872F0008892F0008AD
S315080001508B2F00088D2F00088F2F0008912F00087D
S31508000160932F0008952F0008972F0008992F00084D
S315080001709B2F00089D2F00089F2F0008A12F00081D
S31508000180A32F0008A52F000810B5054C237833B90E
S31508000190044B13B10448AFF300800123237010BD4C
S315080001A0500100200000000024730008084B10B519
S315080001B01BB108490848AFF300800848036803B92B
S315080001C010BD074B002BFBD0BDE81040184700BFF9
S315080001D0000000005401002024730008500100208C
S315080001E000000000154B002B08BF134B9D46A3F5D6
S315080001F0803A00218B460F461348144A121A06F015
S31508000200FFFB0F4B002B00D098470E4B002B00D05E
S3150800021098470020002104000D000D48002802D050
S315080002200C48AFF3008006F0C5FB2000290002F059
S315080002302FFE06F0ABFB00BF0000080000000220FE
S315080002400000000000000000500100204C190020AA
S31508000250000000000000000008B50121054800F074
S3150800026069FE012803D000F005F9012008BD002029
S3150800027008BD00BF0000024008B5642000F0C8F8B9
S3150800028008BD00BF08B500F0C9F808BD30B583B091
S315080002900446154B1B78BBB90121042000F0CAFEA1
S315080002A04FF40063009301258DF804508DF806502D
S315080002B000238DF8073002238DF8053069460B4870
S315080002C000F0F6FD084B1D70012C05D14FF40061B6
S315080002D0064800F039FE04E04FF40061034800F0D8
S315080002E031FE03B030BD00BF6C010020000802409B
S315080002F0704700BF704700BF00B5C7B04FF48C7297
S315080003000021684606F07CFB69460A4806F002F8B2
S3150800031038B9009B3BB19DF8083013F0100F04D094
S3150800032004E0002002E0002000E0012047B05DF86C
S3150800033004FB00BF2C6A0008004870472C6A0008B6
S3150800034008B50748002380F828320A22054905F02F
S3150800035063FC18B90122024B83F8282208BD00BFA6
S31508000360700100204C6A000810B50D4B93F828322E
S31508000370012B02D10A4805F007FF03F0E5FA00F160
S31508000380640403E003F0E0FA844205D340210548FB
S3150800039000F064FF0028F5D0034805F0E1FF10BD22
S315080003A070010020004400402C6A000808B5044B80
S315080003B093F82832012B02D1014805F0E5FE08BD65
S315080003C07001002010B504460F4B93F82832012B14
S315080003D015D10D4906F04CF8002810DA0A48002312
S315080003E080F8283205F0D0FE09E0084800F02EFF14
S315080003F08021064800F032FF0028F9D00134217820
S315080004000029F2D110BD00BF700100200044004051
S31508000410014B1880704700BF9C03002008B503F005
S3150800042093FA104B1B6898421AD30F4B1B7843B9A3
S3150800043001220D4B1A704FF480510C4800F084FDD0
S3150800044007E00022084B1A704FF48051074800F065
S3150800045079FD03F079FA064B1B881844014B18609E
S3150800046008BD00BFA0030020A40300200008024026
S315080004709C03002008B54FF48051024800F062FD45
S3150800048008BD00BF00080240024A137843F0010382
S31508000490137070470000002030B587B0154D002155
S315080004A0284600F033FE0024ADF804404FF482736A
S315080004B0ADF80630ADF80840ADF80A40ADF80C4086
S315080004C04FF40073ADF80E30ADF81040ADF8124099
S315080004D00723ADF8143001A9284600F0F1FD21469E
S315080004E0284600F027FE0121284600F00FFE07B037
S315080004F030BD00BF0038004070B582B0214D4FF4C2
S315080005008051284600F01EFD02238DF80530012390
S315080005108DF8043000248DF807408DF806404FF416
S31508000520004602A941F8086D284600F0C1FC31468C
S31508000530284600F007FD10E00221134800F008FEE7
S315080005400028F9D0FF21104800F0F2FD01210E48DD
S3150800055000F0FEFD0028F9D00134092CECD94FF43F
S315080005600043009302238DF804308DF805300022ED
S315080005708DF806208DF807306946024800F098FC89
S3150800058002B070BD00040240003800402DE9F04179
S3150800059088B00121022000F04DFD01214FF4804072
S315080005A000F064FD4FF48058CDF8048002268DF8DB
S315080005B0096001278DF8087000248DF80B408DF826
S315080005C00A40294D01A9284600F072FC41462846F2
S315080005D000F0B8FC05220D21284600F0B7FC0522DC
S315080005E00E21284600F0B2FC05220F21284600F00D
S315080005F0ADFC4FF4604301938DF808608DF80960EF
S315080006008DF80A408DF80B6001A9284600F050FCC9
S31508000610ADF80C404FF48273ADF80E30ADF81040CB
S31508000620ADF81240ADF814404FF40073ADF816302B
S315080006303023ADF81830ADF81A400723ADF81C3052
S31508000640A5F5E63503A9284600F03AFD21462846D1
S3150800065000F070FD3946284600F058FDFFF74CFFBC
S3150800066008B0BDE8F08100BF0004024008B50146A5
S31508000670064800F05DFD0121044800F069FD0028E8
S31508000680F9D0024800F050FDC0B208BD003800405D
S3150800069038B503F059F900F5FA75FF20FFF7E6FFBC
S315080006A00446FF2803D003F04FF98542F5D8FF2CFE
S315080006B014BF0020012038BD08B54FF48051034807
S315080006C000F040FCFF20FFF7D1FF08BD0004024000
S315080006D010B54FF48051084800F036FCFF20FFF7AC
S315080006E0C5FFFFF7D5FF18B90446FFF7E5FF00E099
S315080006F00124204610BD00BF0004024038B5044658
S315080007000D4610F0800F07D000F07F040021372037
S31508000710FFF7F4FF012831D8FFF7CEFFFFF7D8FF20
S3150800072058B344F04000FFF7A1FF280EFFF79EFFDD
S31508000730C5F30740FFF79AFFC5F30720FFF796FFB3
S31508000740E8B2FFF793FF0CB1012000E09520082CD2
S3150800075000D18720FFF78AFF0C2C02D1FF20FFF774
S3150800076085FF0A24FF20FFF781FF10F0800F05D0D0
S31508000770631E13F0FF04F5D138BDFF2038BD00BF56
S3150800078010B50446FF20FFF771FF207010BD00BFAB
S31508000790F8B505460E4603F0D7F800F16407FF20C2
S315080007A0FFF764FF0446FF2803D103F0CDF887421C
S315080007B0F5D8FE2C11D16C1C2846FFF7E1FF204620
S315080007C00235FFF7DDFF023EF5D1FF20FFF74EFFAA
S315080007D0FF20FFF74BFF0120F8BD0020F8BD00BF42
S315080007E070B505460C46FFF753FF034618B3204677
S315080007F0FFF73CFFFD2C1BD04FF400762C4614F86F
S31508000800020BFFF733FF6878FFF730FF2546023EF5
S31508000810F4D1FF20FFF72AFFFF20FFF727FFFF206D
S31508000820FFF724FF00F01F00052803D0002302E08D
S31508000830012300E00123184670BD00BF002840F0E0
S31508000840A380534B1B7813F0020F03D0504B187834
S31508000850C0B2704770B582B0FFF798FE4FF480516A
S315080008604C4800F071FB00210846FFF747FF0128B6
S315080008706AD103F069F800F57A754FF4D571082046
S31508000880FFF73CFF01283FD109E0FF20FFF7EEFE06
S3150800089002AB234403F8040C0134E4B200E000245C
S315080008A0032CF2D99DF80630012B4FD19DF807305D
S315080008B0AA2B4DD103F048F8854206D94FF080415E
S315080008C0A920FFF71BFF0028F4D103F03DF8854265
S315080008D040D900213A20FFF711FF58B1002440E023
S315080008E0FF20FFF7C3FE02AB234403F8040C0134D0
S315080008F0E4B200E00024032CF2D99DF8043013F08A
S31508000900400F29D00C242CE00021A920FFF7F6FE81
S31508000910012802D80224A92601E00124264603F06C
S3150800092013F8854205D900213046FFF7E7FE00286F
S31508000930F5D103F009F8854210D94FF4007110205B
S31508000940FFF7DCFE60B90CE000240AE0002408E0AA
S31508000950002406E0002404E0042402E0002400E069
S3150800096000240D4B1C60FFF7A7FE3CB1084A13781C
S3150800097003F0FE031370FFF78FFD01E0FFF784FD18
S31508000980034B1878C0B201E00120704702B070BD71
S315080009900000002000040240A803002018B9034BF9
S315080009A01878C0B270470120704700BF00000020C9
S315080009B0B8BB38B50D461C46ABB31D4B1B7813F0B8
S315080009C0010F32D11B4B1B6813F0080F00D15202DE
S315080009D0012C0BD111461120FFF790FED8B94FF420
S315080009E000712846FFF7D4FEA0B914E0114612207C
S315080009F0FFF784FE78B94FF400712846FFF7C8FE62
S31508000A0018B105F50075013CF5D100210C20FFF75A
S31508000A1075FE00E00024FFF74FFE201C18BF0120DA
S31508000A2038BD04207047042038BD032038BD00BFF8
S31508000A3000000020A8030020002846D170B50D4606
S31508000A4016461C46002B42D0244B1B7813F0010F88
S31508000A503FD1224B1B7813F0040F3CD1204B1B6867
S31508000A6013F0080F00D15602012C0AD1314618207E
S31508000A70FFF744FE18BBFE212846FFF7B1FED8B99A
S31508000A801DE013F0060F03D021469720FFF736FE28
S31508000A9031461920FFF732FE88B9FC212846FFF7B0
S31508000AA09FFE18B105F50075013CF6D1FD21002021
S31508000AB0FFF796FE10B102E0002400E00124FFF7DC
S31508000AC0FBFD201C18BF012070BD042070470420C0
S31508000AD070BD032070BD022070BD00BF000000205D
S31508000AE0A8030020002840F02D81994B1B7813F0AD
S31508000AF0010F40F0298130B585B014460E2900F261
S31508000B000281DFE811F00F00160000015E00000107
S31508000B1000010001000100010001B900BE00CC007F
S31508000B20D900EC00FFF7D4FD002840F0EE80012440
S31508000B3004E100210920FFF7E1FD002840F0E780E5
S31508000B4010216846FFF724FE002800F0E2809DF891
S31508000B5000309B09012B10D19DF809309DF808201B
S31508000B6003EB02229DF807301B0403F47C1313449D
S31508000B7001339B0223600024E0E09DF805209DF8E0
S31508000B800A109DF809305B0002F00F0202EBD11241
S31508000B9003F0060313440233DBB29DF808109DF8F0
S31508000BA00720920002EB91119DF80620920202F4AA
S31508000BB040620A440132093B02FA03F32360002427
S31508000BC0BCE0644B1B6813F0040F21D000218D2074
S31508000BD0FFF794FD002840F09E80FF20FFF746FDB2
S31508000BE010216846FFF7D4FD38B90124A6E0FF2096
S31508000BF0FFF73CFD013DEDB200E03025002DF6D1B2
S31508000C009DF80A301A09102393402360002495E0C2
S31508000C1000210920FFF772FD00287ED110216846C1
S31508000C20FFF7B6FD00287AD04A4B1B6813F0020F6F
S31508000C3011D09DF80A305B0003F07E039DF80B2067
S31508000C4003EBD21301339DF80D209209013A934024
S31508000C502360002472E09DF80A30C3F384019DF8EE
S31508000C600B30DA0002F0180202EB5312531C01FB98
S31508000C7003332360002461E0364B1B68137000249D
S31508000C805CE000210920FFF739FD002849D1102131
S31508000C902046FFF77DFD002845D101244EE00021BE
S31508000CA00A20FFF72BFD00283FD110212046FFF729
S31508000CB06FFDE0BB012441E000213A20FFF71EFD4D
S31508000CC040B101243AE0FF20FFF7D0FC605501351A
S31508000CD0EDB200E00025032DF5D900242EE01D4BCA
S31508000CE01B6813F0040F24D000218D20FFF706FDA2
S31508000CF008BBFF20FFF7BAFC40212046FFF748FD56
S31508000D00D8B901241AE0042418E0002416E00124C6
S31508000D1014E0012412E0012410E001240EE001246D
S31508000D200CE001240AE0002408E0012406E000247F
S31508000D3004E0012402E0012400E00024FFF7BCFCE3
S31508000D40204603E0042070470320704705B030BDF5
S31508000D5000000020A8030020054B1B69002B05DABC
S31508000D60034B044A5A6002F188325A60704700BF42
S31508000D70003C024023016745024A136943F00043D9
S31508000D8013617047003C0240014BD860704700BFB2
S31508000D90003C02400E4BDB6813F4803F10D10C4B2D
S31508000DA0DB6813F0100F0DD1094BDB6813F0EF0F5A
S31508000DB00AD1074BDB6813F0020F07D007207047EC
S31508000DC001207047052070470620704708207047A5
S31508000DD0003C024000B583B008238DF80730FFF7C2
S31508000DE0D9FF8DF8070003E0FFF7D4FF8DF8070059
S31508000DF09DF80730DBB2012BF6D09DF8070003B04B
S31508000E005DF804FB70B5054631B1012906D0022903
S31508000E1007D14FF4007606E0002604E04FF480760A
S31508000E2001E04FF44076FFF7D5FF08281ED1104C95
S31508000E30236923F44073236123691E4326612369CA
S31508000E4023F0F803236123691D4345F00205256154
S31508000E50236943F480332361FFF7BCFF236923F03A
S31508000E6002032361236923F0F803236170BD00BFE1
S31508000E70003C024070B505460E46FFF7ABFF082852
S31508000E8013D10A4C236923F440732361236943F47D
S31508000E9000732361236943F0010323612E60FFF782
S31508000EA099FF236923F00103236170BD003C0240CA
S31508000EB070B400233AE001229A400C68A24334D168
S31508000EC004685D000322AA40D24314400460066801
S31508000ED00C79AC40344304600C79013CE4B2012C33
S31508000EE015D884682240826084684A79AA402243D9
S31508000EF0826046689AB20124944026EA0404446053
S31508000F0046688C7904FA02F292B232434260C468A7
S31508000F109AB256000322B24024EA0202C260C668A8
S31508000F20CC7904FA05F23243C26001330F2BC2D9D9
S31508000F3070BC70470369194201D001207047002030
S31508000F40704700BF018370474183704730B401F092
S31508000F5007039B009A40C908083150F821400F251D
S31508000F6005FA03F324EA030340F8213050F8213048
S31508000F701A4340F8212030BC704700BF10B4294BF3
S31508000F809B6803F00C03042B05D0082B06D053BB33
S31508000F90254B036029E0254B036026E0214B5A6860
S31508000FA05B6803F03F0312F4800F09D01F4AB2FBB7
S31508000FB0F3F21C4B5B68C3F3881303FB02F208E0E9
S31508000FC0194AB2FBF3F3174A5168C1F3881101FBBA
S31508000FD003F2144B5B68C3F3014301335B00B2FBB6
S31508000FE0F3F3036001E0104B03600E4CA368C3F3F0
S31508000FF003130F49CB5CDAB20368D3404360A26897
S31508001000C2F382228A5CD2B223FA02F28260A26812
S31508001010C2F342328A5CD2B2D340C3605DF8044B55
S31508001020704700BF003802400024F40000127A001E
S315080010300400002021B1054B1A6B10431863704752
S31508001040024A136B23EA0000106370470038024017
S3150800105021B1054B5A6B104358637047024A536BCC
S3150800106023EA0000506370470038024021B1054B5F
S315080010701A6C104318647047024A136C23EA00007E
S31508001080106470470038024021B1054B5A6C104372
S3150800109058647047024A536C23EA0000506470474C
S315080010A00038024021B1054B1A6A1043186270478E
S315080010B0024A136A23EA00001062704700380240A9
S315080010C02DE9F041038803F441570D884E888C8832
S315080010D0B1F806800A89B1F80AC08B89B1F80EE022
S315080010E03543254348EA050414434CEA04021A43E7
S315080010F04EEA02033B430380838B9BB223F40063CF
S315080011009BB283830B8A0382BDE8F08129B10388E9
S315080011109BB243F040030380704703889BB223F0D9
S3150800112040039BB203807047808980B2704700BF36
S315080011308181704729B103889BB243F40053038029
S31508001140704703889BB223F400539BB20380704711
S315080011500389194201D0012070470020704700BF5B
S3150800116030B585B004460D46038A9BB223F4405336
S31508001170CA881343038283899BB223F4B05323F0AE
S315080011800C01A8882A896B89024313430B43A38160
S31508001190A38A9BB223F44073AA891343A3826846A1
S315080011A0FFF7ECFE204B9C4203D003F580639C427C
S315080011B001D1039A00E0029AA38913F4004F08D0DC
S315080011C002EB820202EB820229684900B2FBF1F1C6
S315080011D007E002EB820202EB820229688900B2FB71
S315080011E0F1F1124BA3FB01235B091B011A096420C9
S315080011F000FB1212A18911F4004F08D0D200323236
S315080012000A49A1FB0212C2F342121A4307E012016D
S3150800121032320649A1FB0212C2F343121A4392B2B2
S31508001220228105B030BD00BF001001401F85EB517B
S3150800123029B183899BB243F400538381704783891C
S315080012409BB223F400539BB283817047C1F3080114
S31508001250818070478088C0F3080070470388194268
S3150800126001D0012070470020704700BF82B00023DC
S31508001270019300932A4A136843F480331360284B7A
S315080012801B6803F400330093019B01330193009B11
S315080012901BB9019BB3F5A06FF1D1214B1B6813F461
S315080012A0003F02D00123009301E000230093009B36
S315080012B0012B32D11A4B1A6C42F080521A64194922
S315080012C00A6842F440420A609A689A609A6842F448
S315080012D000429A609A6842F4A0529A60124A5A608A
S315080012E01A6842F080721A600D4B1B6813F0007F73
S315080012F0FAD040F205620D4B1A60A3F580639A682E
S3150800130022F003029A609A6842F002029A60044B3D
S315080013109B6803F00C03082BF9D102B0704700BF95
S31508001320003802400070004008544007003C024064
S3150800133010B5104CD4F8883043F47003C4F88830DC
S315080013400D4B1A6842F001021A60002199601A686A
S3150800135022F0847222F480321A60084A5A601A68A7
S3150800136022F480221A60D960FFF780FF4FF00063ED
S31508001370A36010BD00ED00E00038024010300024E4
S315080013800369024A12685A6000207047081800204C
S3150800139010B50446D0F8E8351B699847032384F846
S315080013A01231002010BD00BF08B590F8123180F840
S315080013B01331042380F81231D0F8E835DB689847F2
S315080013C0002008BD08B5D0F8E435DB6903B19847B5
S315080013D0002008BD08B5D0F8E4351B6A98470020F8
S315080013E008BD00BF08B5D0F8E4355B6A9847002009
S315080013F008BD00BF10B50446D0F8E8355B699847C4
S31508001400012384F81531002010BD00BF10B504462D
S31508001410D0F8E8359B699847D4F8E4355B6800212D
S3150800142020469847002084F8150110BD10B50446DB
S3150800143000234022194601F0A3F800234022802108
S31508001440204601F09DF8012384F81231D4F8E835D6
S315080014505B68A0789847002010BD00BF10B582B021
S315080014600446694600F06EF99DF8001001F01F0366
S31508001470012B08D013B1022B0AD00EE0694620468C
S3150800148000F0D4FA0EE06946204600F0F3FA09E0C7
S315080014906946204600F00AFB04E001F08001204678
S315080014A001F00CF9002002B010BD00BF10B50446CB
S315080014B0002947D190F81131022B38D1D0F83821BC
S315080014C0D0F824319A4211D9D21AC0F83821C178F5
S315080014D0012904D1D0F828110B44C0F8283192B25A
S315080014E0D4F82811204600F0B5F820E0D0F83C11D1
S315080014F0B1FBF3F203FB121262B98B420AD8D0F899
S315080015004031994206D2114600F0A4F80023C4F8E7
S3150800151040310CE0D4F8E435DB682BB194F812219D
S31508001520032A01D120469847204600F0B3F894F8DC
S315080015301631012B11D12046FFF722FF002384F82C
S3150800154016310AE00A46D0F8E4355B692BB190F803
S315080015501211032901D111469847002010BD00BF7A
S3150800156010B5044659BB90F81131032B32D1D0F887
S315080015709033D0F87C23934214D99B1AC0F8903341
S31508001580C178012904D1D0F880131144C0F880131A
S315080015909A4228BF1A4692B2D4F88013204600F021
S315080015A061F817E0D0F8E4351B6923B190F81221E9
S315080015B0032A00D19847204600F05CF80AE00A465C
S315080015C0D0F8E4359B692BB190F81211032901D1A3
S315080015D011469847002010BDF8B504460D46164634
S315080015E01F4601F0E5FCC4F8E475069BC4F8E83527
S315080015F0C4F8EC652946204600F074FFD4F8E835AF
S315080016001B689847204601F025FDF8BD10B504462D
S31508001610D0F8E4351B689847D4F8E8359B689847AE
S31508001620002010BD08B5D0F8E4355B68984700205F
S3150800163008BD00BF10B504461346C4F83C21C4F8DB
S315080016403821022280F811210A46002101F012F8F9
S31508001650002010BD08B513460A46002101F00AF815
S31508001660002008BD08B513460A46002100F0D4FF3D
S31508001670002008BD10B50446042380F81131002364
S315080016801A46194600F0F6FF204600F009FF00202A
S3150800169010BD00BF10B50446052380F8113100239C
S315080016A01A46194600F0B8FF204600F0F9FE002059
S315080016B010BD00BF0346002002E00130C0B201336E
S315080016C01A78002AF9D1704710B504464B88012BC1
S315080016D009D1C0F81831D0F8E4359B6898472046F8
S315080016E0FFF7C8FF10BD022B29D18B8813F0FF0F17
S315080016F025D1026952681B0A013B042B17D8DFE87B
S3150800170003F003070B0F1300012363F306120EE021
S31508001710022363F306120AE0032363F3061206E0C4
S31508001720042363F3061202E0052363F30612044B4F
S315080017301A60012384F816312046FFF79BFF10BD77
S315080017400818002090F8CC350B7090F8CD354B7002
S3150800175090F8CE3590F8CF2503EB02234B8090F80E
S31508001760D03590F8D12503EB02238B8090F8D2353B
S3150800177090F8D32503EB02239BB2CB80C0F8403107
S31508001780012380F81131704710B50446802100F016
S3150800179095FF0021204600F091FF204600F080FECC
S315080017A010BD00BF30B583B005460C464A88130AFB
S315080017B0013B062B67D8DFE803F004162266665E4F
S315080017C06200D0F8EC351B680DF106018078984761
S315080017D0E388402B03D095F81231012B57D1082303
S315080017E0ADF8063053E0D0F8E4359B6A0DF10601F2
S315080017F08078984702234370C5F8F00547E0D2B2CF
S31508001800052A34D8DFE802F0030B131B232BD0F884
S31508001810EC355B680DF106018078984737E0D0F81B
S31508001820EC359B680DF10601807898472FE0D0F8D3
S31508001830EC35DB680DF106018078984727E0D0F88B
S31508001840EC351B690DF10601807898471FE0D0F842
S31508001850EC355B690DF106018078984717E0D0F8FA
S31508001860EC359B690DF10601807898470FE0214613
S31508001870FFF78AFF19E02146FFF786FF15E02146A4
S31508001880FFF782FF11E02146FFF77EFF0DE0BDF866
S31508001890063053B1E28842B19A4228BF1A46ADF8DB
S315080018A0062001462846FFF7C5FE03B030BD00BF37
S315080018B038B504468B88E3B9CB88D3B98D7805F05B
S315080018C07F0590F81231032B02D1FFF75DFF38BD73
S315080018D080F81451294600F035FF2046FFF7CAFE66
S315080018E01DB1022384F8123138BD012384F8123160
S315080018F038BD2046FFF748FF38BD00BF10B504467F
S315080019008B78214A1370012B02D9FFF73DFF10BDD2
S3150800191090F81221022A02D0032A10D030E05BB1D7
S3150800192080F81031032280F812211946FFF76EFE5F
S315080019302046FFF79FFE10BDFFF79CFE10BD5BB962
S31508001940022280F8122180F810311946FFF76AFE44
S315080019502046FFF78FFE10BD90F810118B420CD071
S31508001960FFF760FE084B197884F810112046FFF738
S315080019704DFE2046FFF77EFE10BDFFF77BFE10BD2D
S31508001980FFF702FF10BD00BFB003002008B5CB88E3
S31508001990012B02D0FFF7F8FE08BD90F81231022B92
S315080019A002D0032B05D00AE001220649FFF742FEC2
S315080019B008BD012200F58871FFF73CFE08BDFFF758
S315080019C0E3FE08BDB803002008B590F81231023BC3
S315080019D0012B0DD80122084B1A60D0F8183113B123
S315080019E00322054B1A6002220349FFF723FE08BDAE
S315080019F0FFF7CAFE08BD00BFAC03002010B50446B9
S31508001A0090F81231023B012B0DD84B88012B0CD1D3
S31508001A100023C0F81831D0F8E4359B68984720466B
S31508001A20FFF728FE10BDFFF7AFFE10BD08B54B78CF
S31508001A30092B1BD8DFE803F011171A141A08051A20
S31508001A400E0BFFF7AFFE13E0FFF732FF10E0FFF7CC
S31508001A5055FF0DE0FFF79AFF0AE0FFF7B5FF07E02D
S31508001A60FFF732FE04E0FFF7C9FF01E0FFF78CFE3F
S31508001A70002008BD38B504460D4690F81231032BF0
S31508001A800FD10B79012B09D8D0F8E4359B68984714
S31508001A90EB8843B92046FFF7EDFD04E0FFF774FE37
S31508001AA001E0FFF771FE002038BD00BF38B50546D6
S31508001AB00C468A88D1B26378012B27D0002B49D0EF
S31508001AC0032B40F0818090F81231022B02D0032BB1
S31508001AD007D017E0002977D0802975D000F0EEFDF1
S31508001AE072E0638823B919B1802901D000F0E6FDB8
S31508001AF0D5F8E4359B682146284698472846FFF7D7
S31508001B00B9FD61E02146FFF73FFE5DE090F812312E
S31508001B10022B02D0032B07D018E0002954D08029C5
S31508001B2052D000F0CBFD4FE06388002B4CD149B171
S31508001B30802907D000F0E4FDD5F8E4359B682146F6
S31508001B40284698472846FFF795FD3DE02146FFF7CA
S31508001B501BFE39E090F81231022B02D0032B06D077
S31508001B602FE089B380292FD000F0A8FD2CE052B2CF
S31508001B70002A10DA01F07F0101EB8101CB00034452
S31508001B8093F81E311BB10122104B1A6013E0002294
S31508001B900E4B1A600FE0002A0DDB01EB8101CB002A
S31508001BA0034493F876331BB10122084B1A6002E00E
S31508001BB00022064B1A60022204492846FFF73AFD1E
S31508001BC002E02146FFF7E0FD002038BDB4030020FF
S31508001BD0D0B170B50D4616460446FFF76BFD0130C9
S31508001BE0400080B23080287003236B70022307E020
S31508001BF05A1CD2B20134E9540233DBB20021A9548B
S31508001C0021780029F4D170BD704700BFC3684FF032
S31508001C10FF325A60C3686FF080425A61014BC2684E
S31508001C20936170470008008030B583B005460024EC
S31508001C300194032001F010FAEB681A690192013445
S31508001C400E4A944217D8019A002AF2DA019A42F00B
S31508001C5001020192019A1A610023EA681269019247
S31508001C600133064A934203D8019A12F0010FF4D1C0
S31508001C70032001F0F1F9002003B030BD400D030048
S31508001C8010B4C4786CB903339B10323200EB82006F
S31508001C908468002203E051F8040B206001329A425E
S31508001CA0F9D300205DF8044B704700BF10B4033227
S31508001CB09210D0F8D040002303E0206841F8040BC6
S31508001CC001339342F9D308465DF8044B704700BFC9
S31508001CD030B40023C3700123837040238380012915
S31508001CE00DD10123C37208230370042343704FF4F4
S31508001CF0A073C380022303724FF0A0440CE051B9CD
S31508001D000023C3720C230370062343704FF4A063A9
S31508001D10C380234C00E00024C46004F5006303611B
S31508001D2000230FE004EB431202F51065191D00EBC2
S31508001D3081018D6002F5306203F1140100EB810127
S31508001D404A60013342789342ECD304F580634361D9
S31508001D5004F58863C0F8CC30002309E004EB43118E
S31508001D6001F5A06103F1220200EB820291600133C2
S31508001D700578AB42F2D3002309E004EB033101F501
S31508001D80805103F1320200EB820291600133AB42CB
S31508001D90F3D304F56064C0F80C41002030BC7047EA
S31508001DA00000044038B50446037A012B22D10025E9
S31508001DB0C268936B6FF31043417A09B143F48013F9
S31508001DC09363E268D3686FF386136FF396536FF3E2
S31508001DD051436FF3D343D3602046FFF725FFE378DB
S31508001DE0012B19D1052363F3440545F02005E36863
S31508001DF09D6011E0C268D16841F04003D360FFF7E7
S31508001E0013FF4FF45023627A0AB14FF4E813E268DD
S31508001E109363142001F02CF9E378012B07D1E368CA
S31508001E209D68052262F3440545F020059D60002063
S31508001E3038BD00BFC268936843F001039360002071
S31508001E40704700BFC268936823F0010393600020BF
S31508001E50704700BF00B583B000230193019A42F092
S31508001E6020020192019A61F38A120192C2680199CD
S31508001E701161C268126901920133074A934203D875
S31508001E80019A12F0200FF4D1032001F0E5F80020A2
S31508001E9003B05DF804FB00BF400D030000B583B036
S31508001EA000230193019A42F010020192C268019937
S31508001EB01161C268126901920133074A934203D835
S31508001EC0019A12F0100FF4D1032001F0C5F8002092
S31508001ED003B05DF804FB00BF400D030008B5C268F7
S31508001EE0D3686FF35D736FF39E73012902D143F0D4
S31508001EF0005302E009B943F08043D360322001F071
S31508001F00B7F8002008BD00BFC368586900F0010093
S31508001F10704700BF08B5FFF7F7FF10F1FF3018BF8D
S31508001F20012008BDC36858699B691840704700BFFF
S31508001F300269136861F301031360704738B50546F3
S31508001F400024C3689C61C3686FF080425A61FFF73A
S31508001F505DFEEB7803B9102444F0804444F4701411
S31508001F6044F4605444F00C04EA68936923EA0403D1
S31508001F701C439461002038BD70B504460025D0F88E
S31508001F800C311D600269136865F3CC231360C37AAC
S31508001F90012B27D12E460321FFF7CAFFE2688023CB
S31508001FA05362202262F31F4563F30F05E1688D62D1
S31508001FB0A02161F30F0663F31F46E368C3F80461C3
S31508001FC04FF4907363F30F0662F31F46E368C3F892
S31508001FD008614FF4A07363F30F066FF31F46E368B7
S31508001FE0C3F80C6110212046FFF734FF2046FFF79F
S31508001FF055FF236900221A6123695A6123694FF044
S31508002000FF3199612369DA6116E0131D04EB830336
S315080020109B681B68002B02DA4FF0904100E0002114
S31508002020131D04EB83039868016099680020086112
S315080020309B68FF219960013263789A42E5D30022B2
S3150800204018E002F1140304EB83035B681B68002B9A
S3150800205002DA4FF0904100E0002102F1140304EB8C
S315080020608303586801605968002008615B68FF218E
S315080020709960013263789A42E3D32269136943F47B
S3150800208080731361E378012B09D10323402262F39D
S315080020908A0343F4803362F3594322691363204663
S315080020A0FFF74CFF002070BD03699B68C3F341032B
S315080020B0022B04D005D8012B03D00320704701203A
S315080020C070470220704700BF03699B6882691168E0
S315080020D0C3F34103022B02D06FF30A0102E0032384
S315080020E063F30A0111600269536843F4807353600D
S315080020F00020704730B400224B78012B08D10D78A8
S315080021002C1D00EB8404A468AB4063F30F0209E0BE
S315080021100D7805F1140400EB840464680123AB40D0
S3150800212063F31F42236813F4004F0DD18D6865F3DE
S315080021300A03CD7865F39343C98861F3995343F04D
S31508002140805343F4004323600369D9690A43DA617B
S31508002150002030BC704700BF70B4002215464B788B
S31508002160012B08D10E78311D00EB81018C68B34034
S3150800217063F30F0509E00B7803F1140400EB8404FC
S3150800218064680121994061F31F456FF3CF322260DD
S315080021900269D36923EA0503D361002070BC70473E
S315080021A038B54B78012B58D10B78043300EB8303F1
S315080021B09B681A681C694B692BB96FF312040123D3
S315080021C063F3DC440DE063F312048D682B44013B92
S315080021D0B3FBF5F363F3DC44CB78012B01D163F34E
S315080021E05E740B78043300EB83039B681C61C37829
S315080021F0012B07D10B78043300EB83039B680C692A
S315080022005C610CE0CB78012B09D04B693BB10C78AB
S31508002210012303FA04F405696B6B23436B63CB78DC
S31508002220012B09D103699B6813F4807F02D142F020
S31508002230005201E042F0805242F004420B78043327
S3150800224000EB83039B681A60CB78012B44D18B8AF9
S315080022500A78C968FFF714FD3EE00B78143300EBE3
S3150800226083035B681A681C694B6933B98B6863F327
S315080022701204012363F3DC440CE08D682B44013B14
S31508002280B3FBF5F3C3F3090363F3DC4405FB03F37C
S3150800229063F312040B78143300EB83035B681C6149
S315080022A0C378012B06D10B78143300EB83035B68E4
S315080022B00C695C61CB78012B06D14B7913B142F0DE
S315080022C0005201E042F0805242F004420B78143387
S315080022D000EB830043681A60002038BD30B482B032
S315080022E04B78012B49D183691A681C6900944C699B
S315080022F06CB99DF800406FF306048DF800409DF810
S315080023000240012565F3C4048DF8024017E08D6884
S31508002310AC4207D94D619DF8004065F306048DF877
S31508002320004005E09DF8005064F306058DF800505E
S315080023309DF80240012565F3C4048DF80240009C0F
S315080023401C61C478012C06D10C78043400EB840493
S31508002350A4680D69656142F004421A60C378002BCF
S315080023604CD14B69002B49D00A78012303FA02F2B3
S3150800237001694B6B13434B6340E00B78143300EB56
S3150800238083035B681A681B6900934B6973B98C6889
S315080023909DF8003064F306038DF800309DF802308E
S315080023A0012464F3C4038DF802300EE08C684C6196
S315080023B09DF8003064F306038DF800309DF802306E
S315080023C0012464F3C4038DF802300B78143300EB50
S315080023D083035B68009C1C61C378012B06D10B78CC
S315080023E0143300EB83035B680C695C6142F00442BA
S315080023F00B78143300EB830043681A60002002B0A0
S3150800240030BC70474B78012B0DD10B78043300EBA9
S31508002410830082681368002B01DA43F0804343F493
S315080024200013136008E00B78143300EB830042684E
S31508002430116841F400131360002070474B78012B94
S3150800244005D10B78043300EB8300806804E00B7831
S31508002450143300EB8300406802686FF35552CB785B
S31508002460023BDBB2012B01D842F080520260002009
S31508002470704700BF03699869DB691840000C70470C
S31508002480143100EB81014B689A680369586910405A
S31508002490704700BF03699869DB69184080B27047C6
S315080024A082B000230093C0238DF803304FF0000359
S315080024B0012262F3C4038DF8023018238DF8003028
S315080024C0436D009A1A61C378012B08D1436D00F257
S315080024D0CC525A61436D1A684FF080221A6002B0D6
S315080024E0704700BF38B50446FFF7F2FB012384F8AE
S315080024F01231002284F8142115E091001144CB0012
S315080025002344012183F81D1183F81C21A3F82221F5
S31508002510002183F81F114020C3F82401C3F82811AD
S31508002520C3F83011013260788242E6D3002214E003
S3150800253091001144CB002344002183F8751383F8D6
S315080025407423A3F87A2383F877134025C3F87C53BA
S31508002550C3F88013C3F8881301328242E8D32046B1
S31508002560FFF770FC2046FFF71DFC00212046FFF709
S31508002570B5FC2046FFF700FD2046FFF75BFC38BD9B
S3150800258070B54DB2002D09DA01F07F0606EB860616
S31508002590F40004F58C740444043408E001F07F0662
S315080025A006EB8606F40004F55C740444043401F072
S315080025B07F012170ED0F6570A260E37005B1E180BF
S315080025C0022B01D1002323712146FFF793FD00203A
S315080025D070BD00BF10B54AB2002A09DA01F07F04BF
S315080025E004EB8404E30003F58C730344043308E026
S315080025F001F07F0404EB8404E30003F55C730344F1
S31508002600043301F07F011970D20F5A701946FFF78B
S31508002610A3FD002010BD00BF70B501F07F04A60021
S315080026203519E9000D4601F55C710144043105448C
S31508002630C5F88023C5F888330023C5F88C3385F898
S31508002640753385F87443C378012B05D104EB8405EB
S31508002650EB000344C3F8842304EB8404E300034437
S3150800266093F8743313B9FFF739FE01E0FFF798FDC5
S31508002670002070BD70B501F07F05AE007119CC0061
S3150800268004F58C740444211D2E44F40004440126E8
S3150800269084F81D6184F81C51C4F82821C4F82C213B
S315080026A00022C4F83421C4F8303115B9FFF716FEF4
S315080026B001E0FFF775FD002070BD00BF10B54AB2F6
S315080026C0002A09DA01F07F0404EB8404E30003F529
S315080026D08C730344043306E001EB8104E30003F53D
S315080026E05C730344043301249C7001F07F01197064
S315080026F0D20F5A701946FFF785FE002010BD00BF9D
S3150800270010B54AB2002A09DA01F07F0404EB840402
S31508002710E30003F58C730344043306E001EB8104FC
S31508002720E30003F55C730344043300249C7001F052
S315080027307F011970D20F5A701946FFF77FFE20469F
S3150800274010BD00BF002361F30A13026911680B4329
S315080027501360704708B50369596841F002025A6068
S31508002760032000F085FC08BD10B50446044B1B6821
S315080027705B6A98474FF08043E2685361012010BDB9
S315080027801400002038B50446C3685D6815F0040FC8
S3150800279003D0044B1B689B6A9847E3685D60012079
S315080027A038BD00BF1400002010B50446837A43B133
S315080027B0D0F80C316FF341036FF30003D0F80C2106
S315080027C013602269536823F001035360054B1B68A5
S315080027D09B69204698474FF00043E2685361012001
S315080027E010BD00BF1400002030B583B00546002494
S315080027F08DF8074090F812318DF80730154B1B6895
S315080028005B6998472B699A684FF40064EB685C61CA
S31508002810AB7AE3B112F0010F19D095F81531012BF7
S3150800282015D19DF80730DBB2032B10D1D5F80C2152
S31508002830136843F001031360D5F80C21136843F0BD
S3150800284003031360044A136943F006031361012066
S3150800285003B030BD1400002000ED00E010B50446BA
S31508002860044B1B68DB6898470823E268536101201C
S3150800287010BD00BF1400002010B50446044B1B68A9
S31508002880DB6998474FF48013E2685361012010BD55
S315080028901400002010B50446044B1B681B6A9847B1
S315080028A04FF40013E2685361012010BD14000020A4
S315080028B010B402691469536BCB40DB01DBB22343C6
S315080028C0043100EB81008268906818405DF8044B7B
S315080028D0704700BF2DE9F0410746FFF7CBFD0446D8
S315080028E0002553E014F0010F4ED05FFA85F84146F3
S315080028F03846FFF7C5FD064610F0010F2BD0012616
S3150800290005F1140307EB83035B689E60FB78B3420B
S3150800291010D105F1140307EB83035B681969AA0054
S315080029202A44D3003B44D3F87C23C1F31201521A3C
S31508002930C3F88C23184B1B681B68414638469847D2
S31508002940FB78012B07D135B997F81131052B02D140
S315080029503846FFF7A5FD16F0020F06D0022605F148
S31508002960140307EB83035B689E6016F0080F0BD011
S31508002970094B1B689B6838469847082605F11403D7
S3150800298007EB83035B689E6001356408002CA9D1B8
S315080029900120BDE8F08100BF140000202DE9F041B8
S315080029A007460D468A000A44D3000344D3F830216B
S315080029B0D3F83411521AD3F824319A4200D8134660
S315080029C003F103084FEA98082B1D07EB83039B685E
S315080029D09B6927E05B1A05EB8501CA003A44D2F8E1
S315080029E02461B34200D81E4606F103084FEA980848
S315080029F0AB002B44DC003C44B3B2EAB2D4F828114D
S31508002A003846FFF73DF9D4F828313344C4F828315D
S31508002A10D4F834311E44C4F834612B1D07EB830304
S31508002A209B689B699BB298450BD2AB002B44DA0096
S31508002A303A44D2F83411D2F83031994201D2002BF7
S31508002A40C8D10120BDE8F0812DE9F0410746FFF71E
S31508002A5021FD044600265EE014F0010F59D05FFA06
S31508002A6086F841463846FFF723FF054610F0010F62
S31508002A701ED0012303FA06F039694A6B22EA0002DE
S31508002A804A631D46321D07EB820292689360244B07
S31508002A901B685B68414638469847FB78AB4207D1C6
S31508002AA036B997F81131042B02D13846FFF7F8FCEE
S31508002AB015F0080F05D00825331D07EB83039B681F
S31508002AC09D6015F0100F05D01025331D07EB830305
S31508002AD09B689D6015F0400F05D04025331D07EB18
S31508002AE083039B689D6015F0020F05D00225331DF0
S31508002AF007EB83039B689D6015F0800F09D031466C
S31508002B003846FFF74BFF8025331D07EB83039B6889
S31508002B109D6001366408002C9ED10120BDE8F08135
S31508002B20140000202DE9F0410546C268936923F098
S31508002B3010039361C3681C6A04F00F06C4F3434389
S31508002B40022B02D0062B1CD02BE047F6F07323424B
S31508002B5027D0C4F30A144FEA860808EB0603DF00F9
S31508002B6007442246D7F88013FFF7A0F8D7F8803332
S31508002B702344C7F88033D7F88C331C44C7F88C43F2
S31508002B800FE0082200F2CC51FFF790F8C4F30A14BC
S31508002B90B2009119CB002B44D3F88C231444C3F804
S31508002BA08C43EA68936943F0100393610120BDE8FA
S31508002BB0F08100BF2DE9F84304460025A8462F46B4
S31508002BC02E460269536823F0010353602946FFF72E
S31508002BD041F92B460CE01A1D04EB82029268FF218C
S31508002BE0916003F1140204EB82025268916001338A
S31508002BF062789342EFD323694FF0FF329A614FF020
S31508002C00010969F30F0569F31F452369DD6148F07A
S31508002C100B082369C3F8148047F00B0723691F6163
S31508002C20226913686FF30A1313602046FFF738FC0E
S31508002C3046F48056E3685E61034B1B681B692046B1
S31508002C4098474846BDE8F8831400002038B504467E
S31508002C50FFF73AFAE368DD682046FFF725FA032806
S31508002C6008D10023A3704FF40073A380092363F3EC
S31508002C708D2506E00123A3704023A380052363F373
S31508002C808D25E368DD604FF40053E2685361012047
S31508002C9038BD00BF2DE9F8430546FFF73BF9002884
S31508002CA06AD02846FFF73EF90646002868D0C0F3E2
S31508002CB0074818F0080F04D02846FFF70BFE04460D
S31508002CC000E0002418F0040F03D02846FFF7BCFEE6
S31508002CD00443F7B217F0020F02D00223EA685361E1
S31508002CE04FEA166919F0800F03D02846FFF75CFDF6
S31508002CF00443C6F3072616F0080F03D02846FFF745
S31508002D0073FD044317F0080F03D02846FFF7A6FD06
S31508002D10044317F0100F03D02846FFF703FF0443B8
S31508002D2016F0100F03D02846FFF744FF044316F0A9
S31508002D30200F03D02846FFF789FF044318F0100F29
S31508002D4003D02846FFF798FD044318F0200F03D058
S31508002D502846FFF79FFD044319F0400F03D0284685
S31508002D60FFF702FD044317F0040F08D02846FFF7C3
S31508002D7009FD2043BDE8F8830020BDE8F883204616
S31508002D80BDE8F8832DE9F04383B001210846FEF734
S31508002D9051F90124009400268DF804608DF8076027
S31508002DA002258DF80550384F69463846FEF780F8F3
S31508002DB021464FF40030FEF759F921462046FEF722
S31508002DC039F9072229463846FEF7C0F807220321B3
S31508002DD03846FEF7BBF88DF806608DF807408DF883
S31508002DE004504FF00408CDF800808DF80550694668
S31508002DF03846FEF75DF88DF804504FF00809CDF80F
S31508002E00009069463846FEF753F821462846FEF7ED
S31508002E1011F907F58067092249463846FEF796F8FC
S31508002E20092211463846FEF791F84FF4407300938D
S31508002E308DF804508DF805508DF806608DF807401A
S31508002E4069463846FEF734F821464FF00070FEF71B
S31508002E500DF921464046FEF7EDF84FF480570097E6
S31508002E608DF804408DF806608DF807408DF80550FA
S31508002E70064C69462046FEF71BF839462046FEF7FB
S31508002E8061F803B0BDE8F083000002400008024084
S31508002E9008B5FFF777FF01F01FF801F02DF8FCE7FA
S31508002EA007498D460749084A084B9A42BEBF51F85A
S31508002EB0040B42F8040BF8E7054880470548004725
S31508002EC00000022030730008000000205001002096
S31508002ED031130008E50100083349344A002301E0AC
S31508002EE041F8043B9142FBD3FFF7D2FFFEE7FEE72A
S31508002EF0FEE7FEE7FEE7FEE7FEE7FEE7FEE7FEE79C
S31508002F00FEE7FEE7FEE7FEE7FEE7FEE7FEE7FEE78B
S31508002F10FEE7FEE7FEE7FEE7FEE7FEE7FEE7FEE77B
S31508002F20FEE7FEE7FEE7FEE7FEE7FEE7FEE7FEE76B
S31508002F30FEE7FEE7FEE7FEE7FEE7FEE7FEE7FEE75B
S31508002F40FEE7FEE7FEE7FEE7FEE7FEE7FEE7FEE74B
S31508002F50FEE7FEE7FEE7FEE7FEE7FEE7FEE7FEE73B
S31508002F60FEE7FEE7FEE7FEE7FEE7FEE7FEE7FEE72B
S31508002F70FEE7FEE7FEE7FEE7FEE7FEE7FEE7FEE71B
S31508002F80FEE7FEE7FEE7FEE7FEE7FEE7FEE7FEE70B
S31508002F90FEE7FEE7FEE7FEE7FEE7FEE7FEE7FEE7FB
S31508002FA0FEE7FEE7FEE70000500100204C1900206E
S31508002FB070B582B001210846FEF73CF84FF4C053BD
S31508002FC0009303268DF8056002238DF8043000254A
S31508002FD08DF806508DF807501D4C69462046FDF7BA
S31508002FE067FF0A220B212046FDF7B0FF0A220C21B3
S31508002FF02046FDF7ABFF01210420FEF71BF84FF42E
S315080030000063009301248DF804408DF806508DF86E
S3150800301007408DF8056005F1804505F502356946D6
S315080030202846FDF745FF6B6923F400636B6121466B
S315080030304FF48040FEF728F821468020FEF708F86E
S3150800304021464FF08050FEF72DF802B070BD00BF44
S3150800305000000240704700BF06E000BF013300E0F1
S3150800306000231B2BF9D91046421E0028F8D17047B9
S3150800307008B54FF47A7303FB00F0FFF7EDFF08BDC0
S3150800308020230B80004870477000002008B590F890
S315080030901231032B01D100F08BFE002008BD00BFC2
S315080030A008B500F085FE002008BD00BF08B5084633
S315080030B000F0B0FE002008BD08B50B7813F0600FCD
S315080030C021D14B780A2B12D00B2B15D0062B1AD1EF
S315080030D04B881B0A212B05D1CA88172A28BF172215
S315080030E00A4901E00A491722FEF7A4FA0BE0012271
S315080030F00849FEF79FFA06E08B7813B9054A13606C
S3150800310001E0FEF741FB002008BD00BF8200002059
S3150800311079000020BC03002010B504468121FFF782
S3150800312059FA01212046FFF755FA002010BD00BFC5
S3150800313010B50446022340228121FFF721FA022313
S31508003140402201212046FFF71BFA4023034A0121AA
S315080031502046FFF761FA002010BD00BF0C190020B9
S31508003160004870470C19002012230B80004870474E
S31508003170B000002004230B8000487047AC000020F4
S3150800318010B5044C0A4621460348FEF721FD2046A1
S3150800319010BD00BF0C1800205C6A000810B5044C6E
S315080031A00A4621460348FEF713FD204610BD00BF18
S315080031B00C180020706A000810B5044C0A4621460F
S315080031C00348FEF705FD204610BD00BF0C18002079
S315080031D0806A000810B5044C0A4621460348FEF7E3
S315080031E0F7FC204610BD00BF0C180020906A0008A6
S315080031F010B5044C0A4621460348FEF7E9FC20466A
S3150800320010BD00BF0C180020986A0008704700BF60
S31508003210704700BF704700BF08B5FDF769F808BDDD
S3150800322008B5FDF767F808BD08B50120FDF72EF8C3
S3150800323008BD00BF08B50020FDF728F808BD00BF87
S31508003240F0B5002421E0134D15F8147005EB44057C
S3150800325095F801E007EB0E0505FB00054AF2104C50
S315080032609CFBF5F605FB16C66EB99CFBF5F5ADB2EB
S315080032700D80013DADB2B5F5806F04D2177083F8A5
S3150800328000E00120F0BD0134E4B2112CDBD90020A6
S31508003290F0BD00BFD86A000800B583B001AB0DF1D8
S315080032A005020DF106014FF4FA70FFF7C9FF012870
S315080032B003D0EE21384800F0D9FD384B00225A6178
S315080032C01A6842F400421A6001E000F0ABFE334B84
S315080032D01B6813F4004FF8D1304B1A6822F002022B
S315080032E01A601A6842F001021A6001E000F09AFEBC
S315080032F02A4B5B6813F0010FF8D09DF805305A1E6B
S315080033009DF80430013B1B0543EA0243BDF806203D
S31508003310013A1343214AD361136823F0010313606A
S3150800332001E000F07FFE1D4B5B6813F0010FF8D13A
S315080033301A4BD3F8002242F00102C3F80022D3F850
S315080033401C2222F00102C3F81C22D3F80C2242F0F8
S315080033500102C3F80C220022C3F84022C3F8442213
S31508003360D3F8042222F00102C3F80422D3F8142267
S3150800337022F00102C3F81422D3F81C2242F00102FB
S31508003380C3F81C22D3F8002222F00102C3F8002257
S3150800339003B05DF804FB00BFB06A00080064004093
S315080033A038B504460D46214B9B6813F0806F04D14F
S315080033B04FF4A2711E4800F059FD1C4BD3F880212A
S315080033C002F00102C3F88021D3F8802142F07C4242
S315080033D042F40012C3F88021C3F88451E178A27838
S315080033E0120442EA0162617842EA012221780A431C
S315080033F0C3F88821E179A279120442EA0162617967
S3150800340042EA012221790A43C3F88C21D3F88021A4
S3150800341042F00102C3F8802101E000F003FE034BED
S315080034209B6813F0806FF8D038BD00BF0064004079
S31508003430B06A0008214BDB6813F0030F3CD01F4B22
S31508003440D3F8B03113F0040F04D11C4BD3F8B031C4
S315080034505B0D05E0194BD3F8B031DB0843F00043A8
S3150800346040F26762934220D1144BD3F8B821027018
S31508003470D3F8B821120A4270D3F8B821120C827018
S31508003480D3F8B821120EC270D3F8BC210271D3F852
S31508003490BC21120A4271D3F8BC21120C8271D3F8EE
S315080034A0BC311B0EC371012000E00020034AD3681B
S315080034B043F02003D3607047002070470064004043
S315080034C008B500F0F7F908BD10B500F003FAA0B189
S315080034D0FCF7C2FE88B100F057FD00F00DFA00F0C7
S315080034E0FDF920F0604020F07F00044B186000F0E2
S315080034F0F5F9446800F0E0F9A04710BD08ED00E0D2
S3150800350070B508E0461C4D1C0B78037000F08AFD68
S31508003510224630462946531E9CB2002AF2D170BD77
S3150800352038B50546002419E000F07CFD04EB44029A
S3150800353093000C4AD358AB420ED804EB44018A00D8
S3150800354008490A44526813449D4205D204EB4400D4
S3150800355083000B44187A38BD0134E4B2092CE3D948
S31508003560FF2038BD2C6B000808B5C1F3080353B912
S315080035700368994209D040F8041B4FF40072FFF71C
S31508003580BFFF012008BD002008BD012008BD00BFFF
S315080035902DE9F04107460068FFF7C2FFFF282ED045
S315080035A0FDF7DAFBF320FDF7EFFBFDF7F3FB012848
S315080035B018D1FDF7E1FB0020BDE8F0813E68A300C5
S315080035C006EB03083B445D6800F02CFD294640469F
S315080035D0FDF750FC08280AD156F824309D4208D138
S315080035E0013400E000247F2CE8D9012402E00024FD
S315080035F000E00024FDF7C0FB2046BDE8F08100206E
S31508003600BDE8F08138B50D460B4B984207D0044605
S315080036100A4B994205D0FFF7BBFF18B908E0084CDA
S3150800362000E0054C29462046FFF79EFF10B938BD35
S31508003630002038BD204638BDC003002000800008A1
S31508003640C40500202DE9F04106460C4617461D46DE
S3150800365021F4FF7828F001080368B3F1FF3F04D18D
S315080036604146FFF781FF034630B33368984505D0D6
S3150800367041463046FFF7C6FF0646D0B13368E41A1E
S315080036803444043400F0CEFC331DE31AB3F5007F4E
S3150800369007D308F500713046FFF7B4FF064650B168
S315080036A0041D17F8013B04F8013B013DEAD101234B
S315080036B002E0002300E000231846BDE8F08100BFC1
S315080036C0884229D838B504460D46012826D90B293B
S315080036D026D8FDF741FBF320FDF756FBFDF75AFB0D
S315080036E0012813D1FDF748FB002038BD00F09AFCED
S315080036F002210C4B33F81400FDF784FB082803D08D
S31508003700FDF73AFB002038BD0134E4B2AC42EDD9EE
S31508003710FDF732FB012038BD00207047002038BD78
S31508003720002038BDFC6A00084FF0FF33024A1360D8
S31508003730024A1360704700BFC4050020C00300207A
S3150800374070B504460D461646FFF7EAFEFF281AD05E
S3150800375060190138FFF7E4FEFF2816D024F4FF733A
S3150800376023F001030A4A934206D12B4632462146E4
S315080037700848FFF767FF70BD2B46324621460648C4
S31508003780FFF760FF70BD002070BD002070BD00BF50
S3150800379000800008C0030020C405002070B5064656
S315080037A00C46FFF7BDFE054630190138FFF7B8FE8F
S315080037B0FF2D06D0FF2806D001462846FFF780FFD2
S315080037C070BD002070BD002070BD00BF114B1B6886
S315080037D0B3F1FF3F18D000B583B00E4B59689A680D
S315080037E01144DA6811441A6911445A6911449A69EC
S315080037F01144DA698B185B4202AA42F8043D042197
S315080038000548FFF79DFF01E00120704703B05DF80A
S3150800381004FB00BFC0030020888100080D4B1A680E
S3150800382004331B6813440C4A126813440B4A126883
S3150800383013440B4A11680B44043212681A44094BA4
S315080038401B681344084A1268D34201D10120704705
S315080038500020704700800008088000080C800008D7
S3150800386010800008188000088881000808B50D4BEC
S315080038701B68B3F1FF3F04D00A48FFF789FE0346E9
S3150800388068B1094B1B68B3F1FF3F05D00648FFF73F
S315080038907FFE034610B902E0012300E00123184623
S315080038A008BD00BFC0030020C405002000487047BB
S315080038B00080000872B6704762B6704708B5FFF711
S315080038C033FF08BD08B5FFF73BFF08BD08B5FFF78E
S315080038D065FF08BD08B5FFF7A1FF08BD08B5FFF7E6
S315080038E0E5FF08BD08B5FFF771FF034610B1FFF7FE
S315080038F0BDFF0346184608BD0022014B1A607047F3
S3150800390010E000E008B5FFF7F7FF054B054A5A60D7
S3150800391000229A6005211960034B1A6008BD00BF92
S3150800392010E000E03F900200C8070020044B1B6827
S3150800393013F4803F03D0034A1368013313607047BA
S3150800394010E000E0C807002008B5FFF7EFFF014BBD
S31508003950186808BDC807002010B504468021094824
S31508003960FDF77CFC58B121460648FDF76FFC80211F
S315080039700448FDF773FC0028F9D0012010BD00208B
S3150800398010BD00BF0044004010B50446202106487B
S31508003990FDF764FC012805D10348FDF75BFC2070A0
S315080039A0012010BD002010BD0044004010B584B0B1
S315080039B04FF4614300930023ADF80430ADF80630A8
S315080039C0ADF80830ADF80C300C23ADF80A30054CCC
S315080039D069462046FDF7C4FB01212046FDF728FC71
S315080039E004B010BD0044004070B506460D46402997
S315080039F003D976210F4800F039FA2846FFF7ACFFBD
S31508003A00012803D07A210B4800F030FA00240CE094
S31508003A1000F008FB305DFFF79FFF012803D08321E4
S31508003A20044800F023FA0134A4B2ABB29C42EFD3A7
S31508003A3070BD00BFA46B000838B5224B1C789CB932
S31508003A402148FFF7A1FF01283AD11F4B1B78002B0D
S31508003A5031D0FFF779FF1D4B186000221C4B1A70F6
S31508003A600122184B1A702BE00546194B1B780133B7
S31508003A7015481844FFF788FF0446012810D1144B4F
S31508003A801A780132D2B21A700F4B1B789A4214D1A7
S31508003A9010492846FFF734FD00220A4B1A700FE03A
S31508003AA0FFF752FF094B1B686433984207D9002475
S31508003AB0044B1C7004E01C4602E0002400E00024CD
S31508003AC0204638BD11080020D0070020CC0700206A
S31508003AD012080020D1070020094B03F11801002223
S31508003AE005E09A745961183318310132D2B2002AA6
S31508003AF0F7D09A7400225A61014A024B1A6070473D
S31508003B0018080020140800200B4B1B6873B110B46A
S31508003B105C69094A146019749860D86000225A745E
S31508003B201860013908445860987C01E0FF20704706
S31508003B305DF8044B704700BF1408002038B50446EA
S31508003B400D46012804D94FF4CD71154800F08EF9B9
S31508003B5062002244D300134A13445A7C1B7C9A42BF
S31508003B601AD062002244D3000E4A1344DA6815704C
S31508003B705A7C01325A74DA680132DA605B689A4212
S31508003B800CD9084A63001819C1000846515803465B
S31508003B901344D960012038BD002038BD012038BD46
S31508003BA0D06B00081808002008B50146024B1878A3
S31508003BB0FFF7C4FF08BD00BFCC08002038B504468F
S31508003BC00D46012804D94FF4DE71144800F04EF969
S31508003BD004EB4402D300124A1344587CE0B1620055
S31508003BE02244D3000E4A13449A6812782A705A7CE3
S31508003BF0013A5A749A6801329A605B689A420AD9FD
S31508003C00074A63001819C100084651580346134469
S31508003C109960012038BD012038BD00BFD06B00086F
S31508003C201808002008B50146024B1878FFF7C6FFAA
S31508003C3008BD00BF4808002010B50446012804D96D
S31508003C404FF4EE71044800F011F904EB4404E30064
S31508003C50024A1344587C10BDD06B0008180800208F
S31508003C6030B583B0FFF738FF0F4C4021601CFFF7D3
S31508003C704BFF20700D4D4021681CFFF745FF28704B
S31508003C802378FF2B01D0FF2803D17921084800F0BB
S31508003C90EDF8084B0093084B084A01210848FDF740
S31508003CA09BFC03B030BD00BFCC08002048080020AC
S31508003CB0D06B0008C40000204400002090000020BB
S31508003CC01009002008B50348FEF744FD0020FCF75C
S31508003CD0DDFA08BD1009002070B506460D463F29D5
S31508003CE003D99A210F4800F0C1F82846FFF75CFF70
S31508003CF0012803D09E210B4800F0B8F800240CE0F8
S31508003D0000F090F9305DFFF74FFF012803D0A72197
S31508003D10044800F0ABF80134A4B2ABB29C42EFD32E
S31508003D2070BD00BFD06B000838B505461B48FEF7C6
S31508003D30B1FF1B4B1C7874B91A48FFF773FF0128AB
S31508003D4029D1184B1B780BB30122154B1A70002288
S31508003D50154B1A701FE0144B1B7801331148184491
S31508003D60FFF760FF0446012812D10F4B1A7801327B
S31508003D70D2B21A700B4B1B789A420BD10B492846C4
S31508003D80FFF7BEFB0022064B1A7004E01C4602E051
S31508003D90002400E00024204638BD00BF100900209A
S31508003DA0440F0020040F00200D090020050F0020F5
S31508003DB030B583B0134B1878FFF73EFF00B30546BE
S31508003DC0402800D94025002412E00DF107010D4BCB
S31508003DD01878FFF7F3FE012804D04FF492710A48C9
S31508003DE000F044F89DF80720084B1A550134E4B250
S31508003DF0A542EAD82B46054A81210548FEF73AFC32
S31508003E0003B030BDCC080020D06B00088C08002019
S31508003E101009002070B500EB8000C300104A134457
S31508003E20B3F88C63002410E00E4B1D78FFF798F961
S31508003E30015D2846FFF782FE012804D040F24311AF
S31508003E40094800F013F80134A4B2B442ECD3FFF7E2
S31508003E5087F94023024601210148FEF7DDFB70BDC4
S31508003E601009002048080020D06B000808B500F0AB
S31508003E70D9F8FCE708B500F0CDF8012816D000F00F
S31508003E805FF998B10A4B1B78012B0FD1FFF75CFD40
S31508003E90084B1B6803F5FA63984207D30022044BC4
S31508003EA01A7000F057F908B9FFF70EFB08BD00BFF6
S31508003EB0450F0020480F002008B50122044B1A7050
S31508003EC0FFF742FD034B1860FFF7D4FF08BD00BF9C
S31508003ED0450F0020480F002008B5FFF7F1FA00F05B
S31508003EE09DF8FFF70FFDFFF7E9FC00F013F900F066
S31508003EF00FF8FFF7E1FF08BD08B500F093F8FFF7E4
S31508003F0015FD00F035FA00F017F8FFF7B3FF08BD06
S31508003F1010B502F0ADFCFFF7BFF9064C012323707C
S31508003F20FFF744FD00232370FFF79AFE0223237050
S31508003F3010BD00BFE000002008B51148FFF77AFA67
S31508003F40012805D101220F4B1A700D4802F0AEFC6C
S31508003F500B48FFF771FD012805D10022094B1A709D
S31508003F60074802F0A3FC0648FFF7DEFE012805D144
S31508003F700222044B1A70024802F098FC08BD00BFE2
S31508003F804C0F0020E000002008B5FFF79BFE08BD97
S31508003F9038B504460D460C4B1B78012B02D1C9B225
S31508003FA0FFF7FEF9084B1B781BB9E9B22046FFF765
S31508003FB01BFD054B1B78022B03D1E9B22046FFF700
S31508003FC08BFE02F06BFC38BDE0000020074B1B7827
S31508003FD0022B05D0032B05D0012B05D040207047B6
S31508003FE03F2070470020704708207047E0000020F7
S31508003FF0074B1B78022B05D0032B05D0012B05D0C8
S31508004000402070473F2070470020704708207047BF
S31508004010E000002008B502F039FC08BD08B5FCF739
S315080040202BF908BD08B5FCF72DF908BD00F00F02FD
S3150800403002F13003092802D902F137007047054A10
S3150800404012681A44527802F00302022A00D1203B71
S31508004050D8B27047E400002038B505460C4600097A
S31508004060FFF7E4FF207005F00F00FFF7DFFF607031
S315080040700023A370204638BD034601310D4AA2FB32
S315080040800323DB08F9D110B400230B70094BA3FBFB
S315080040900023DB081A4603EB83035C00031B30335B
S315080040A001F8013D1046002AF0D108465DF8044B98
S315080040B0704700BFCDCCCCCC30B4002423461EE0DC
S315080040C0025D134909681144497801F00301022980
S315080040D000D1203AD2B2A2F13001C9B2162912D8BB
S315080040E0A2F13A05EDB2062D0FD9092901D9373AB9
S315080040F0D1B21A01D2B20A44D3B20134E4B2012CC5
S31508004100DED9184602E0002000E0002030BC7047E7
S31508004110E400002008B50022054B1A700549064838
S3150800412001F04EFD18B177210448FFF79FFE08BD40
S31508004130CC0F0020F86B0008D80F0020FC6B000895
S31508004140034B1B780BB9012070470020704700BF4E
S31508004150CC0F002008B5FFF75DFF01280AD0084BF1
S315080041601B784BB9FCF7C8F8012807D10122044B84
S315080041701A7008BD002008BD002008BD002008BD33
S31508004180CC0F00200378114A1168CA18527802F039
S315080041900302022A00D1203B532B0DD14378194440
S315080041A04A7812F0040F09D0312B09D0322B09D0E6
S315080041B0332B09D10220704703207047032070472C
S315080041C0002070470120704703207047E400002054
S315080041D070B506460230FFF76FFF054684B204360F
S315080041E03046FFF769FF2844C5B2013CA4B202363F
S315080041F0012CF5D8ED43EDB23046FFF75DFF854259
S3150800420001D0002070BD012070BD00BF2DE9F0412E
S31508004210044616460F4601B120B940F261215348BB
S31508004220FFF724FE2046FFF7ADFF0546032800F0FA
S3150800423093802046FFF7CCFF002800F09080012DE0
S3150800424028D015B1022D52D08DE0A01CFFF734FFFF
S3150800425085B2201DFFF730FF4FEA0028C7F8008017
S31508004260A01DFFF729FF404438600834033D2DB2EE
S3150800427056B92846BDE8F0812046FFF71DFFF055E0
S3150800428002340137BFB200E00027AF42F4DB28460C
S31508004290BDE8F081A01CFFF70FFF85B2201DFFF7D0
S315080042A00BFF4FEA0048C7F80080A01DFFF704FF80
S315080042B008EB0028C7F8008004F10800FFF7FCFEA9
S315080042C0404438600A34043D2DB256B92846BDE844
S315080042D0F0812046FFF7F0FEF05502340137BFB2F1
S315080042E000E00027AF42F4DB2846BDE8F081A01CB9
S315080042F0FFF7E2FE85B2201DFFF7DEFE4FEA0068F3
S31508004300C7F80080A01DFFF7D7FE08EB0048C7F8DE
S31508004310008004F10800FFF7CFFE08EB0028C7F875
S31508004320008004F10A00FFF7C7FE404438600C34E9
S31508004330053D2DB256B92846BDE8F0812046FFF75F
S31508004340BBFEF05502340137BFB200E00027AF428A
S31508004350F4DB2846BDE8F0810020BDE8F0814FF087
S31508004360FF30BDE8F0810020BDE8F081FC6B000855
S3150800437070B5AC4B1B78002B00F0E781012B29D1D7
S31508004380FFF79CFAFBF7DCFFA748FCF71BF8A748E2
S31508004390FCF718F8FBF7D0FF01220146A44801F004
S315080043A03BFC30B1A348FCF70DF80120FBF7FEFFF4
S315080043B070BDA148FCF706F8A048FCF703F8A0482A
S315080043C0FCF700F89F4B00221A605A600222954BB0
S315080043D01A7070BD022B40F0EF809B4C04F50C72EE
S315080043E04FF48071994802F019F894F841326BB18C
S315080043F09048FBF7E7FF0220FBF7D8FF04F50C709F
S3150800440001F0C2FE0022874B1A7070BDB0B18F480A
S31508004410002200F5C071FFF7F9FE0446B0F1FF3F30
S315080044200DD18448FBF7CEFF0320FBF7BFFF80487A
S3150800443001F0AAFE00227B4B1A7070BD0024002CE6
S315080044405BDD804B5B6833B9804BD3F880217D4BAD
S315080044501A605C6051E07D4AD2F88011794A126888
S315080044601A44914203D12344764A536045E0724880
S31508004470FBF7A8FF7648FBF7A5FF764E714D314648
S315080044806868FFF7F9FD3046FBF79CFF7248FBF7B3
S3150800449099FF3146E878FFF7DFFDB11CA878FFF7EA
S315080044A0DBFD311D6878FFF7D7FDB11D2878FFF7CA
S315080044B0D3FD3046FBF786FF6848FBF783FF69683C
S315080044C02868FFF703FA60B95A48FBF77BFF05200F
S315080044D0FBF76CFF564801F057FE0022514B1A7045
S315080044E070BD5548FBF76EFF5548FBF76BFF574BFA
S315080044F0D3F88021534B1A605C60534BD3F844229F
S31508004500D3F83C329A4240F020810021484801F015
S315080045104DFE60B14748FBF755FF0420FBF746FF01
S31508004520434801F031FE00223E4B1A7070BD454BE0
S315080045305B68002B39D04048FBF744FF4448FBF73B
S3150800454041FF444D3F4C29466068FFF795FD2846D4
S31508004550FBF738FF4048FBF735FF2946E078FFF7B9
S315080045607BFDA91CA078FFF777FD291D6078FFF76A
S3150800457073FDA91D2078FFF76FFD2846FBF722FF7C
S315080045803648FBF71FFF61682068FFF79FF960B997
S315080045902848FBF717FF0520FBF708FF244801F01A
S315080045A0F3FD00221F4B1A7070BD2348FBF70AFF64
S315080045B003221C4B1A7070BD032B40F0C680224C98
S315080045C004F50C724FF48071204801F027FF94F827
S315080045D041326BB12248FBF7F5FE0220FBF7E6FEF7
S315080045E004F50C7001F0D0FD00220E4B1A7070BD58
S315080045F0002839D0154800F5807200F5C071FFF71C
S3150800460005FE0546B0F1FF3F2FD11648FBF7DAFE47
S315080046100320FBF7CBFE064801F0B6FD0022014B4E
S315080046201A7070BDCC0F0020186C00083C6C00088E
S3150800463008120020646C00086C6C0008746C000892
S31508004640986C0008D00F0020D80F002030140020E6
S31508004650C86C00088C0F0020D46C0008786D000820
S31508004660F06C0008146D00080025002D40DD374861
S31508004670FBF7A8FE364C21462846FFF7FDFC2046E8
S31508004680FBF7A0FE3348FBF79DFE334E214696F80E
S315080046908301FFF7E1FCA11C96F88201FFF7DCFC19
S315080046A0211D96F88101FFF7D7FCA11D96F8800118
S315080046B0FFF7D2FC2046FBF785FE2848FBF782FE6B
S315080046C006F580722946D6F88001FFF7FBF860B92F
S315080046D02348FBF777FE0620FBF768FE214801F022
S315080046E053FD0022204B1A7070BD2048FBF76AFE66
S315080046F01F4BD3F84422D3F83C329A4225D11D48A1
S31508004700FBF760FEFFF7EEF860B91548FBF75AFEAF
S315080047100720FBF74BFE134801F036FD0022124B2B
S315080047201A7070BD1148FBF74DFE1348FBF74AFE99
S315080047300C4801F029FD1148FBF744FE00220A4BFC
S315080047401A70FBF711FEFEF7BFFE70BD386D000844
S315080047508C0F0020486D000830140020786D000882
S31508004760646C000808120020CC0F00206C6C00084E
S31508004770D80F0020606D00087C6D0008946D000855
S315080047804278007840EA0220704700BFC2788378F2
S3150800479043EA0222437843EA0223007840EA0320E8
S315080047A0704700BF0170090A417070470170C1F374
S315080047B007234370C1F307438370090EC17070471E
S315080047C013462AB10A78027001300131013BF9D14A
S315080047D0704700BF01700130013AFBD1704700BF36
S315080047E030B4451C037808781B1A013A04D04C1CCF
S315080047F028462146002BF4D0184630BC704700BF27
S3150800480000E0013003780BB18B42FAD118467047A5
S3150800481002394369023B994204D24389806A01FB03
S31508004820030070470020704770B506460D4601F133
S315080048301A00FFF7A5FF04463378032B05D105F1C7
S315080048401400FFF79DFF44EA004070BD70B50646A8
S315080048500C46154691B204F11A00FFF7A3FF337808
S31508004860032B04D1290C04F11400FFF79BFF70BD3C
S315080048702DE9F04180460F4601F11A00FFF780FF47
S3150800488050BB3D7805F03F056B1E03EB430503EB74
S3150800489085050126002411E0174B185D3844FFF7FB
S315080048A06FFF36B1FE2D1AD828F8150006460135D1
S315080048B003E04FF6FF73984214D101340C2CEBD960
S315080048C03B7813F0400F10D0FE2D11D8002328F89E
S315080048D015300120BDE8F0810020BDE8F0810020F8
S315080048E0BDE8F0810020BDE8F0810120BDE8F08137
S315080048F00020BDE8F08100BF546E00082DE9F8439A
S3150800490080460F4691464B730F23CB7200240C73D7
S31508004910214607F11A00FFF745FF09F1FF3303EBBC
S31508004920430603EB860625464FF6FF739D4202D0E3
S3150800493038F8165001360C4B185D29463844FFF7EF
S3150800494031FF0DB94FF6FF7501340C2CECD94FF633
S31508004950FF739D4202D038F816300BB949F040096A
S3150800496087F80090BDE8F883546E000870B582B0E9
S31508004970054616461C460B22FFF722FF052C12D8C1
S3150800498014E0023600220CE003F0010101EB4404B6
S315080049905B0814F4803F03D084F4883484F021043F
S315080049A001320F2AF0D93388002BEAD1072300E019
S315080049B0134604F00F0202F13001392901D902F138
S315080049C037015A1E02A8034403F8081C2409EFD12C
S315080049D07E210346134403F8081C002300E0013334
S315080049E0934202D2E95C2029F9D1591C2B44072AA3
S315080049F005D802A8104410F8080C013200E020205F
S31508004A0018700B460729F0D902B070BD0B21002398
S31508004A10DA0142EA5303027852FA83F3DBB2013031
S31508004A200139F5D118467047016821B94FF0FF33AF
S31508004A3016E0013200E00A4613781F2B01D93A2BFB
S31508004A40F7D13A2B0BD110B44C1C0B78303B092B01
S31508004A5008D8A24209D15BB9013202600AE00023F4
S31508004A60184670474FF0FF3304E04FF0FF3301E07C
S31508004A704FF0FF3318465DF8044B704738B50C46BF
S31508004A8070B1054603685BB11A784AB1D98882883D
S31508004A90914205D15878FBF781FF10F0010F03D03A
S31508004AA000232360092038BD2B682360002038BD09
S31508004AB0F8B5C37803B30446C66A00F13007012384
S31508004AC0324639464078FBF7B7FFB8B90023E3709A
S31508004AD0236AF31AA269934212D2A57808E0A36959
S31508004AE01E440123324639466078FBF7A5FF013D8F
S31508004AF0012DF4D80020F8BD0020F8BD0120F8BD2E
S31508004B000020F8BD70B5C36A8B4212D004460D4624
S31508004B10FFF7CEFF064668B901232A4604F130019D
S31508004B206078FBF745FF10B101264FF0FF35E562C7
S31508004B3000E00026304670BD10B504460023C37059
S31508004B404FF0FF33C362FFF7DDFFD8B904F22E201A
S31508004B50FFF716FE4AF65523984215D104F166006A
S31508004B60FFF714FE20F07F400A4B98420ED004F15E
S31508004B708200FFF70BFE20F07F40064B984207D1D4
S31508004B80002010BD042010BD032010BD002010BD5C
S31508004B90022010BD464154002DE9F04784B00E4668
S31508004BA0174600230B60FFF73FFF051EC0F22C8156
S31508004BB0AA4B53F82540002C00F02881346007F0F2
S31508004BC0FE07237873B16078FBF7E8FE10F0010F53
S31508004BD008D1002F00F01C8110F0040F40F01A8154
S31508004BE0002038E100232370E8B26070FBF726FE48
S31508004BF010F0010F40F010811FB110F0040F40F0C3
S31508004C000D8100212046FFF797FF022815D00026C0
S31508004C1028E004F130002B0103F5DF73184403790B
S31508004C201BB10830FFF7B2FD00E0002004AB03EB30
S31508004C30850343F8100C013500E00025032DE8D95B
S31508004C40002504AB03EB850353F8106C26B13146F7
S31508004C502046FFF771FF00E00320012802D901353D
S31508004C60032DEED9042800F0DB80012800F2DA8053
S31508004C7004F13B00FFF784FDB0F5007F40F0D480D7
S31508004C8004F14600FFF77CFD804620B904F1540084
S31508004C90FFF77CFD8046C4F8188094F8409084F8A5
S31508004CA0029009F1FF33DBB2012B00F2BF8008FB4B
S31508004CB009F994F83D506581002D00F0B9806B1E06
S31508004CC01D4240F0B78004F14100FFF759FD8246C6
S31508004CD0208110F00F0F40F0AF8004F14300FFF77A
S31508004CE04FFD074620B904F15000FFF74FFD074670
S31508004CF004F13E00FFF744FD0346002800F09E80BD
S31508004D0009EB000202EB1A129742C0F09980BF1A0B
S31508004D10B7FBF5F5002D00F0958040F6F5718D424C
S31508004D2001D8012700E002274FF6F5718D4200D918
S31508004D30032702356561E661334423623244A26281
S31508004D40032F0FD104F15A00FFF71AFD00287BD173
S31508004D50BAF1000F7AD104F15C00FFF717FD606223
S31508004D60AD000EE0BAF1000F72D04B446362022F19
S31508004D7001D16D0005E005EB450305F0010505EBDE
S31508004D80530505F2FF15B8EB552F63D34FF0FF33E4
S31508004D902361E36080232371032F2CD104F1600083
S31508004DA0FFF7EEFC012826D1711C2046FFF7AAFE64
S31508004DB008BB0023237104F22E20FFF7E1FC4AF614
S31508004DC05523984217D104F13000FFF7DFFC244B36
S31508004DD0984210D104F50570FFF7D8FC214B98428C
S31508004DE009D104F50670FFF7D1FC206104F50770B8
S31508004DF0FFF7CCFCE06027701B4A138801339BB28F
S31508004E001380E380002026E00B2024E00C2022E01B
S31508004E10002020E00A201EE003201CE00A201AE0F9
S31508004E20012018E00D2016E00D2014E00D2012E0F8
S31508004E300D2010E00D200EE00D200CE00D200AE0FC
S31508004E400D2008E00D2006E00D2004E00D2002E00C
S31508004E500D2000E00D2004B0BDE8F087B81700204B
S31508004E605252614172724161B4170020F8B5066862
S31508004E70012951D97369994250D20C463378022BCD
S31508004E802AD0032B37D0012B4AD101EB5105316AC1
S31508004E9001EB55213046FFF735FE002842D16F1C3D
S31508004EA0C5F30805354495F83050316A01EB5721AA
S31508004EB03046FFF727FE002837D1C7F308073E44D8
S31508004EC096F8300045EA002014F0010F01D00009D9
S31508004ED0F8BDC0F30B00F8BD316A01EB142130466A
S31508004EE0FFF710FE20BB600000F4FF70303030443E
S31508004EF0FFF746FCF8BD316A01EBD4113046FFF7DF
S31508004F0001FEC0B9A00000F4FE7030303044FFF74F
S31508004F103DFC20F07040F8BD0120F8BD0120F8BD29
S31508004F200120F8BD4FF0FF30F8BD4FF0FF30F8BD57
S31508004F304FF0FF30F8BD4FF0FF30F8BD2DE9F041D6
S31508004F400768B1F5001F3DD206460C4611F01F0F43
S31508004F503BD1316185681DB93B78022B00D97D6A42
S31508004F6035B93B89B3EB541F32D97B6AB3611AE072
S31508004F70B7F80A804FEA48280EE029463046FFF778
S31508004F8075FF0546B0F1FF3F25D0012826D97B6974
S31508004F90984226D2C8EB04044445EED22946384640
S31508004FA0FFF736FCB0617561B369EBB103EB5423C7
S31508004FB0B36107F13003C4F308042344F361002006
S31508004FC0BDE8F0810220BDE8F0810220BDE8F0814D
S31508004FD00220BDE8F0810120BDE8F0810220BDE88D
S31508004FE0F0810220BDE8F0810220BDE8F08100BF13
S31508004FF02DE9F843012977D94369994276D21746AC
S315080050000C4605460378022B42D0032B52D0012BBF
S315080050106ED101EB5108016A01EB5821FFF772FDC9
S315080050200646002865D108F10109C8F3080814F0F6
S31508005030010409D005EB080393F8303003F00F0399
S3150800504043EA0713DBB200E0FBB2A84488F8303025
S315080050500123EB70296A01EB59212846FFF752FD17
S315080050600646002845D1C9F3080914B1C7F3071243
S3150800507008E005EB090393F8303023F00F03C7F374
S3150800508003221A43A94489F830200123EB7030E043
S31508005090016A01EB1421FFF735FD064648BB60009F
S315080050A000F4FF703030B9B22844FFF77BFB0123C8
S315080050B0EB701EE0016A01EBD411FFF723FD0646EB
S315080050C0B8B927F07047A40004F4FE7430342C44B1
S315080050D02046FFF75BFB00F0704139432046FFF797
S315080050E065FB0123EB7004E0022602E0022600E0DD
S315080050F002263046BDE8F8832DE9F04107460668E2
S31508005100884629B9F5687DB173699D420ED20EE0CD
S31508005110FFF7ACFE012846D9B0F1FF3F51D07369BD
S3150800512098424ED3454602E0012500E001252C466B
S31508005130013473699C4202D3012D37D902242146D2
S315080051403846FFF793FE38B1012832D0B0F1FF3F59
S3150800515031D0AC42ECD130E04FF0FF322146304638
S31508005160FFF746FF034640B9B8F1000F05D02246BF
S3150800517041463046FFF73CFF034673B9F46033698E
S315080051807269023A934201D2013B3361337943F0A3
S31508005190010333712046BDE8F081012B10D14FF091
S315080051A0FF30BDE8F0810120BDE8F0810020BDE8B0
S315080051B0F081BDE8F081BDE8F0810020BDE8F0810E
S315080051C00120BDE8F08100BFF8B50E460468012944
S315080051D02CD90746114663699E4229D22AB14FF057
S315080051E0FF322046FFF704FF20BB31463846FFF75B
S315080051F03DFE0546F8B101281FD0B0F1FF3F1ED08D
S31508005200002231462046FFF7F3FED0B92369B3F1F1
S31508005210FF3F05D001332361237943F0010323714E
S3150800522063692E469D42E0D30020F8BD0220F8BDF2
S315080052300220F8BDF8BD0020F8BD0220F8BD012007
S31508005240F8BDF8BD2DE9F8430668036903F12005A2
S315080052508369002B6ED0B5F5001F6ED288460446CA
S31508005260C5F30807002F5DD101338361416941B950
S315080052703389B3EB551F55D8002383610420BDE855
S31508005280F8837389013B13EA55234BD1FFF7EEFDEB
S315080052908146012854D9B0F1FF3F54D0736998422A
S315080052A039D3B8F1000F04D10023A3610420BDE867
S315080052B0F88361692046FFF71FFF8146002845D01D
S315080052C0012846D0B0F1FF3F46D03046FFF7F0FB45
S315080052D0002844D14FF40072002106F13000FFF790
S315080052E079FA49463046FFF793FAF0624FF000081C
S315080052F00AE00123F3703046FFF7DAFB90BB08F1AA
S315080053000108F36A0133F36273899845F1D3F36AA6
S31508005310C8EB0303F362C4F8149049463046FFF716
S3150800532077FAA061256107F130084644E661002056
S31508005330BDE8F8830420BDE8F8830420BDE8F883B7
S315080053400220BDE8F8830120BDE8F8830720BDE800
S31508005350F8830220BDE8F8830120BDE8F883012020
S31508005360BDE8F8830120BDE8F88300BFF8B5044618
S315080053700F4606680021FFF7E1FD0246B8B9002589
S31508005380A1693046FFF7BEFB024680B9E3691B7880
S31508005390E52B00D01BB90135BD4201D107E0002538
S315080053A001212046FFF74EFF02460028E8D0042ACE
S315080053B000D107221046F8BD2DE9F8430446884671
S315080053C007684FF0FF094E4604254CE03846FFF7BC
S315080053D099FB054600284BD1E1690A78002A46D090
S315080053E0CB7A03F03F03A371E52A2BD02E2A2BD0C4
S315080053F023F02000082814BF00200120404525D1AD
S315080054000F2B15D112F0400F06D091F80D9002F02F
S31508005410BF02236963621646B24219D14B7B99458E
S3150800542018D1A06AFFF724FAB0B1013EF6B214E02B
S3150800543026B90846FFF7EAFA814519D04FF0FF3337
S31508005440636215E0FF2608E0FF2606E0FF2604E073
S31508005450FF2602E0FF2600E0FF2600212046FFF790
S31508005460F1FE054620B9A1690029AFD100E004255F
S315080054700DB10023A3612846BDE8F88370B504463C
S3150800548005680669416AB1F1FF3F03D0FFF756FD8B
S31508005490034600E00023BBB9A1692846FFF732FBA3
S315080054A0034670B9E269E52111700122EA702269A2
S315080054B0964206D900212046FFF7C4FE0346002877
S315080054C0EAD0042B00D10223184670BD2DE9F04F0F
S315080054D083B006468A46D1F80090856A002423469A
S315080054E05F1C19F803001F2805D92F2803D05C284C
S315080054F00AD100E0013709EB070219F807302F2B0C
S31508005500F8D05C2BF6D017E0FE2C00F2E2800121E1
S3150800551000F0D6FF8046002800F0DD807F2806D8F8
S3150800552001467148FFF76CF9002840F0D68025F847
S3150800553014803B460134D3E7CAF800201F2802D856
S315080055404FF004080CE04FF0000809E004F10043AE
S31508005550013B35F81330202B01D02E2B02D1013C0C
S31508005560002CF3D1002325F81430002C00F0B78066
S315080055700B222021306AFFF72DF9002300E00133C2
S3150800558035F81320202AFAD02E2AF8D01BB148F075
S31508005590030800E0013C6CB104F10042013A35F819
S315080055A012202E2AF6D14FF0080B4FF0000ACDF83C
S315080055B004A005E04FF0080B4FF0000ACDF804A050
S315080055C003F1010935F81370002F57D0202F03D0A7
S315080055D02E2F05D14C4503D048F003084B46EFE77C
S315080055E0DA4501D24C4515D1BBF10B0F02D148F073
S315080055F0030843E04C4501D048F003084C453DD329
S31508005600019B9B00DBB2019323464FF00B0B4FF037
S31508005610080AD5E77F2F0BD90021384600F050FF3E
S31508005620074618B1A0F18007304BDF5D48F0020845
S3150800563027B139462E48FFF7E3F818B148F00308B2
S315080056405F2714E0A7F141039BB2192B04D8019BED
S3150800565043F0020301930AE0A7F161039BB2192BF9
S3150800566005D8019B43F001030193203FBFB2336A7B
S3150800567003F80A704B460AF1010AA1E7336A1A7859
S31508005680E52A01D105221A70BBF1080F03D1019B47
S315080056909B00DBB20193019901F00C020C2A03D09E
S315080056A001F00303032B01D148F0020818F0020F9A
S315080056B00AD1019B03F00303012B01D148F010081E
S315080056C0042A01D148F00808336A83F80B800020C1
S315080056D006E0062004E0062002E0062000E0062098
S315080056E003B0BDE8F08F00BFC06D0008D46D000898
S315080056F0CC6D0008F8B500238B758369002B69D03B
S315080057000D460646436AB3F1FF3F17D0836A002465
S3150800571009E0002100F0D4FE50B1FE2C0AD82A195F
S3150800572090753B4601349F1C18880028F1D102E089
S31508005730002400E000242C440023A375AC7D00223D
S31508005740134628E0F069591CC35C202B22D0052B90
S3150800575000D1E523092907D114B9A8182E2787757A
S31508005760A8182E2747720132A81843728CB9A3F1DC
S315080057704100C0B219280AD8F069007B082901D966
S31508005780102700E00827074201D02033DBB2A8180B
S31508005790837501320B460A2BD4D934B9AB180021CC
S315080057A09975F3691B7B03B90A462A440023537289
S315080057B0F369DB7A2B72F0691C30FEF7E7FF286085
S315080057C0F0691830FEF7DCFFA880F0691630FEF79E
S315080057D0D7FFE880F8BD00BF2DE9F0478146884627
S315080057E001F11A00FEF7CCFFA8BB98F8005005F0A7
S315080057F03F056B1E03EB430503EB850501270024D4
S315080058001BE01F4B185D4044FEF7BAFF06467FB102
S31508005810FE2D23D800F072FE074605F1010A39F875
S31508005820150000F06BFE87421BD13746554603E04C
S315080058304FF6FF73984217D101340C2CE1D998F82A
S31508005840003013F0400F12D0A7B139F81530A3B9BC
S315080058500120BDE8F0870020BDE8F0870020BDE8FC
S31508005860F0870020BDE8F0870020BDE8F08701201A
S31508005870BDE8F0870120BDE8F0870020BDE8F08785
S31508005880546E00082DE9F8430446D0F8008000213C
S31508005890FFF754FB00285CD14FF0FF3363624FF0EB
S315080058A0FF094F46A1694046FFF72CF9064600282E
S315080058B051D1E5692B78002B4FD0E97A01F03F02E8
S315080058C0A271E52B04D011F0080F06D00F2A04D0D8
S315080058D04FF0FF336362FF2733E00F2A17D1A06A20
S315080058E078B313F0400F06D095F80D9003F0BF0378
S315080058F0226962621F46BB421ED16B7B99451DD148
S315080059002946FFF769FFD8B1013FFFB219E027B969
S315080059102846FFF77BF8814522D0216ACB7A13F017
S31508005920010F04D10B222846FEF75AFFD8B14FF0D3
S31508005930FF336362FF2704E0FF2702E0FF2700E04A
S31508005940FF2700212046FFF77DFC0028AAD0BDE8E6
S31508005950F883BDE8F883BDE8F8830420BDE8F8833A
S315080059603046BDE8F8833046BDE8F88330B583B0E5
S3150800597004460191056801E001330193019B1A78F9
S315080059802F2AF9D05C2AF7D00022A2601B781F2B99
S3150800599008D8236A8022DA7200212046FFF7CEFA59
S315080059A0034626E001A92046FFF790FD034600BB03
S315080059B02046FFF767FF236ADA7A034628B10428E8
S315080059C017D112F0040F11D013E012F0040F10D102
S315080059D0A37913F0100F0BD02169C1F308013031F8
S315080059E029442846FEF720FFA060DBE7052300E0F0
S315080059F00523184603B030BD2DE9F04784B0066884
S31508005A00D0F820A0D0F828809AF80B3013F0A00F11
S31508005A1040F08380002400E0013438F81430002B6D
S31508005A20FAD105460C22514601A8FEF7C9FE9DF893
S31508005A300F3013F0010F1ED000238AF80B30AB622B
S31508005A4001270BE03B46424601A95046FEF78EFF6A
S31508005A502846FFF717FF814610B90137632FF1D99A
S31508005A60642F5CD0B9F1040F5BD19DF80F308AF82A
S31508005A700B30C5F828809DF80F3013F0020F06D0BA
S31508005A800C342B4BA3FB0434A408013400E0012496
S31508005A9021462846FFF76AFC034618BB013C21D07D
S31508005AA02969A1EB44112846FFF748FA0346C8B905
S31508005AB0286AFEF7ABFF0746A9693046FFF722F8C2
S31508005AC0034678B93B46E2B2E969A86AFEF716FFCB
S31508005AD00123F37000212846FFF7B4FB034608B9F3
S31508005AE0013CE9D1FBB9A9693046FFF70BF88146B5
S31508005AF0D8B920220021E869FEF76CFE0B22296A34
S31508005B00E869FEF75DFEEA692B6ADB7A03F018039B
S31508005B1013730123F370484607E0062005E00720C3
S31508005B2003E0484601E01846FFE704B0BDE8F08701
S31508005B304FECC44E70B50446FEF7BAFF054600287A
S31508005B4037D12378032B2DD12379012B2AD104F1C0
S31508005B5030064FF4007200213046FEF73BFE4AF647
S31508005B60552104F22E20FEF71DFE13493046FEF796
S31508005B701DFE124904F50570FEF718FE216904F5A5
S31508005B800670FEF713FEE16804F50770FEF70EFED1
S31508005B90E2690132E262012331466078FAF74CFF86
S31508005BA000232371002211466078FAF79BFF00B1A3
S31508005BB00125284670BD00BF52526141727241618B
S31508005BC010B584B001900091144604A840F8041D4D
S31508005BD0FEF72AFF002816DB0E4B53F820300BB1D0
S31508005BE000221A70019B0BB100221A70019B094A08
S31508005BF042F820304BB1012C09D1002201A9684690
S31508005C00FEF7CAFF04E00B2002E0002000E00020B7
S31508005C1004B010BDB81700202DE9F04393B00191E8
S31508005C20002800F0AA80054616460023036002F005
S31508005C301F073A4606A901A8FEF7AEFF002840F05E
S31508005C409E80069B079303AB0F934F4B11930199C5
S31508005C5007A8FFF78BFE044628B90F9B93F90B306C
S31508005C60002B00DA062416F01C0F53D044B1042C7E
S31508005C7003D107A8FFF7C0FE044647F008070BE064
S31508005C809DF8223013F0110F03D116F0040F02D13C
S31508005C9002E0072400E00824002C4BD117F0080F77
S31508005CA048D03A4E31460E980E30FEF77FFD314603
S31508005CB00E981630FEF77AFD20220E9BDA72069EA3
S31508005CC0DDF8388041463046FEF7AEFD81460022B3
S31508005CD041463046FEF7BAFD00210E981C30FEF705
S31508005CE065FD0122069BDA70B9F1000F22D0069BEA
S31508005CF0DE6A0022494607A8FFF766FA0446C8B9CD
S31508005D0031460698FEF7FEFE044609F1FF33069A69
S31508005D10D3600FE074B99DF8223013F0100F06D146
S31508005D2016F0020F06D013F0010F02D102E0042488
S31508005D3000E007244CB917F0080F01D047F02007F8
S31508005D40069BDB6A2B620E9B6B62CCB9069EDDF85E
S31508005D50388041463046FEF767FDA86008F11C000A
S31508005D60FEF714FDE86000236B746B61EB612F741A
S31508005D702E60F388AB80204603E0092001E000E0AE
S31508005D80204613B0BDE8F083B41500200000614832
S31508005D902DE9F04F83B00446884615461F46002372
S31508005DA03B6001A9FEF76AFE002840F0A280607CED
S31508005DB0002840F0A080237C13F0010F00F09A80A1
S31508005DC0E6686369F61AAE42C0F08E802E468BE00E
S31508005DD06369C3F30802002A70D1019A5289013A0D
S31508005DE012EA532912D10BB9A06803E0A16920462B
S31508005DF0FFF73CF8012802D8022060747BE0B0F176
S31508005E00FF3F02D10120607475E0A061DDF804A0AF
S31508005E10A1695046FEF7FCFC054610B902206074DD
S31508005E2069E04D445FEA562B25D009EB0B03BAF817
S31508005E300A20934201D9C9EB020B5B462A46414622
S31508005E409AF80100FAF7B4FD10B10120607452E027
S31508005E50237C13F0400F0BD0E069401B834507D91C
S31508005E604FF4007204F1280108EB4020FEF7A8FC65
S31508005E704FEA4B2530E0E26995421ED0237C13F0A9
S31508005E80400F0ED0012304F128019AF80100FAF711
S31508005E90D3FD10B1012060742DE0237C23F040036C
S31508005EA0237401232A4604F1280101984078FAF759
S31508005EB07FFD10B1012060741DE0E5616169C1F3E1
S31508005EC00801C1F50075AE4200D2354628312A468A
S31508005ED021444046FEF774FCA84463692B44636179
S31508005EE03B682B443B60761B002E7FF471AF002085
S31508005EF001E000E0072003B0BDE8F08F2DE9F04F80
S31508005F0083B00446884616461F4600233B6001A90F
S31508005F10FEF7B4FD002840F0BE80607C002840F003
S31508005F20BC80237C13F0020F00F0B6806369F3424D
S31508005F30C0F0A880DE43A5E06369C3F30802002A1F
S31508005F4040F08180019A5289013A12EA53291DD1FB
S31508005F5033B9A06840B900212046FFF7CDF803E021
S31508005F60A1692046FFF7C8F8002800F08E800128AE
S31508005F7002D10220607490E0B0F1FF3F02D1012007
S31508005F8060748AE0A061A36803B9A060237C13F05B
S31508005F90400F0FD00123E26904F1280101984078E7
S31508005FA0FAF74AFD10B10120607476E0237C23F0ED
S31508005FB040032374DDF804A0A1695046FEF728FCC7
S31508005FC0054610B90220607467E04D445FEA562B17
S31508005FD025D009EB0B03BAF80A20934201D9C9EB7D
S31508005FE0020B5B462A4641469AF80100FAF724FD59
S31508005FF010B10120607450E0E169491B8B450BD94B
S315080060004FF4007208EB412104F12800FEF7D8FB93
S31508006010237C23F0400323744FEA4B2525E0E369EC
S315080060209D420FD06269E3689A420BD201232A4641
S3150800603004F128019AF80100FAF7BAFC10B1012018
S3150800604060742AE0E5616069C0F30800C0F5007570
S31508006050AE4200D2354628302A4641462044FEF74D
S31508006060AFFB237C43F040032374A84463692B44A5
S315080060706361E268934238BF1346E3603B682B448A
S315080060803B60761B002E7FF457AF237C43F020033A
S315080060902374002001E000E0072003B0BDE8F08F7C
S315080060A070B582B004460E460A2902D10D21FFF7C3
S315080060B0F7FF6368002B16DB5D1C23441E733C2D1B
S315080060C00DDD01AB2A4604F10C012068FFF716FF27
S315080060D0019B9D4201D1002501E04FF0FF35656027
S315080060E0A3680133A36002B070BD00BF30B583B0AA
S315080060F0044601A9FEF7C2FC00283CD1227C12F016
S31508006100200F39D012F0400F0CD00123E26904F1B8
S31508006110280101984078FAF78FFC70BB237C23F09E
S3150800612040032374216A0198FEF7ECFC38BB656AC4
S31508006130EB7A43F02003EB72A26829462068FEF743
S3150800614085FBE16805F11C00FEF730FB0D4905F1FA
S315080061501600FEF72BFB002105F11200FEF722FBC5
S315080061600122019BDA700198FFF7E4FC237C23F0F7
S315080061702003237403E002E001E00120FFE703B0F7
S3150800618030BD00BF0000614810B582B00446FFF775
S31508006190ADFF034638B901A92046FEF76FFC034652
S315080061A008B900222260184602B010BDF0B583B0C7
S315080061B004460E4601A9FEF761FC002840F0A480BB
S315080061C0657C002D40F0A180E368B34204D2227CAE
S315080061D012F0020F00D11E46636900226261002E8A
S315080061E05DD0019A57897F026BB1721EB2FBF7F236
S315080061F0013BB3FBF7F18A4205D37A421340636148
S31508006200F61AA16912E0A16879B92046FEF774FF6B
S315080062100146012802D10220607479E0B0F1FF3FFF
S3150800622002D10120607473E0A060A16119BB002649
S3150800623038E0237C13F0020F05D02046FEF75CFFFA
S31508006240014620B91AE02046FEF710FE0146B1F1D4
S31508006250FF3F02D1012060745AE0012903D9019B4E
S315080062605B69994202D30220607451E0A1616369B7
S315080062703B446361F61BBE42DBD800E03E466369D9
S3150800628033446361C6F308035BB10198FEF7C0FAAD
S3150800629010B9022060743BE000EB562602E00026A7
S315080062A000E000266369C3F3080313B3E269964264
S315080062B01FD0237C13F0400F0ED0012304F12801D0
S315080062C001984078FAF7B8FB10B1012060741FE016
S315080062D0237C23F0400323740123324604F128016A
S315080062E001984078FAF764FB10B1012060740FE05A
S315080062F0E6616369E268934209D9E360237C43F067
S3150800630020032374284603E002E0284600E02846D6
S3150800631003B0F0BD30B591B001900D46002205A935
S3150800632001A8FEF739FC0446A8B902AB0D930B4B3E
S315080063300F93019905A8FFF719FB044658B90D9B59
S3150800634093F90B30002B05DB2DB1294605A8FFF77D
S31508006350D1F900E00624204611B030BDB41500205E
S3150800636070B59CB00190022205A901A8FEF714FC9D
S31508006370059B1193044600284AD102AB1993264B74
S315080063801B93019911A8FFF7F1FA044600283FD19B
S31508006390199B93F90B30002B05DB9DF84A3013F057
S315080063A0010F02D102E0062400E00724ECB9059E9D
S315080063B018993046FEF738FA05469DF84A3013F024
S315080063C0100F13D006960890002106A8FEF7B6FD12
S315080063D0044658B9002106A8FEF7EEFF034600B9A1
S315080063E00723042B02D01C4600E0002584B911A817
S315080063F0FFF744F8044630B92DB10022294611A802
S31508006400FEF7E2FE04461CB90598FFF793FB04461F
S3150800641020461CB070BD00BFB41500202DE9F04120
S3150800642082B080460E4617460546002412E06B46A3
S31508006430012201A93846FFF7ABFC009B012B0ED1C0
S315080064409DF804300D2B05D06A1C2B7001340A2BDD
S3150800645004D01546731E9C42E9DB00E0154600236E
S315080064602B700CB9184600E0404602B0BDE8F08132
S3150800647010B594B00446019100230293039303E0F8
S31508006480013401A8FFF70CFE21780029F8D1029AF9
S31508006490002A0BDB6B4604A90198FFF72FFD40B9CC
S315080064A0009B029A9A4207D1039807E04FF0FF3003
S315080064B004E04FF0FF3001E04FF0FF3014B010BD9C
S315080064C07F2817D979B1FF2813D8A0F180030A4A83
S315080064D032F813007047084A32F81320904205D064
S315080064E001339BB200E000237F2BF4D98033D8B266
S315080064F070470020704700BF14710008F0B4B0F56B
S31508006500805F01D2204B02E0204B00E02B461A8820
S31508006510002A36D0904234D31D1D5B88190ADBB297
S315080065209C18A04228DA08292BD8DFE801F00509CB
S315080065300F1215181B1E2100861A35F8160020E0C2
S31508006540821A02F00103C01A80B21AE0103880B22B
S3150800655017E0203880B214E0303880B211E01A38DB
S3150800656080B20EE0083080B20BE0503880B208E006
S31508006570A0F5E35080B204E00029C7D105EB430338
S31508006580C5E7F0BC704700BF206F0008646E0008BE
S3150800659010B4002304E010F8011B0B44DBB22146BB
S315080065A04C1E0029F7D1136001205DF8044B704793
S315080065B00022014B5A707047BC170020034BFE227D
S315080065C0DA7018710222A3F844207047BC1700201D
S315080065D010B5054C00232370FFF7EAFFFF23E3708D
S315080065E00123A4F8443010BDBC170020064BFF2237
S315080065F0DA7000221A71597859719A71DA711A7219
S315080066000622A3F844207047BC17002008B50020CE
S31508006610FFF7D4FF08BD00BF084BFF22DA70084A0F
S315080066209A6400221A715A719A710721D9711A72DD
S315080066305A729A720822A3F844207047BC170020A1
S3150800664014720008044BFF22DA7042689A64012229
S31508006650A3F84420704700BFBC17002010B5084CAB
S31508006660FF23E370E21D4168A06CFFF791FF2071DC
S3150800667000236371A3710823A4F8443010BD00BF3A
S31508006680BC17002008B53120FFF798FF08BD00BFEA
S3150800669038B5084CFF23E370002525716571FDF7B1
S315080066A095FCA071E571257265720723A4F844303C
S315080066B038BD00BFBC17002038B5FDF741FD18B935
S315080066C01020FFF77BFF38BDFFF772FF0D4C012541
S315080066D02570FF23E3701023237100236371FDF7F0
S315080066E075FCA071FDF784FCE071FDF781FCC0F331
S315080066F0072020726572A5720823A4F84430FDF7B6
S31508006700DDF838BDBC17002038B505464478FDF7D6
S315080067105DFC0138844203DD2220FFF74FFF38BDB8
S31508006720084C6A78A16C201DFCF7EAFEFF23E3708B
S315080067306B78A26C1344A3646B780133A4F84430D5
S3150800674038BD00BFBC17002038B504464578FDF7AC
S315080067503DFC0138854203DD2220FFF72FFF38BDB7
S315080067606168084DA9646278281DFCF7C9FEFF23F5
S31508006770EB706378AA6C1344AB6463780133A5F8AD
S31508006780443038BDBC17002038B505460D4B9C6C07
S31508006790FDF71CFC6A1C411E2046FDF793F818B944
S315080067A03120FFF70BFF38BD064CFF23E370FDF7DA
S315080067B00DFC0138A36C1844A0640123A4F84430E6
S315080067C038BD00BFBC17002038B504464578FDF72C
S315080067D0FDFB0238854203DD2220FFF7EFFE38BDB8
S315080067E00F4BFF22DA700122A3F84420617831B9F1
S315080067F0FDF778F890B93120FFF7E0FE38BDA21C06
S31508006800074B986CFDF75EF818B93120FFF7D6FEEE
S3150800681038BD6378024A916C0B44936438BD00BF57
S31508006820BC17002008B54168074B986CFDF74EF871
S3150800683018B93120FFF7C2FE08BD034BFF22DA70F4
S315080068400122A3F8442008BDBC17002008B5FCF7B0
S315080068503BFE034BFF22DA700122A3F8442008BD51
S31508006860BC17002008B589B2FDF792FB08BD00BF2A
S31508006870054B00221A709A6483F84320A3F8442033
S315080068809A705A70704700BFBC170020024B1878E0
S3150800689000B10120704700BFBC1700200022024B40
S315080068A083F84320704700BFBC17002008B503785B
S315080068B0FF2B02D1FFF700FF50E0334A1278012A76
S315080068C060D1C93B352B46D8DFE803F0334545424E
S315080068D045453F363C394545454545454545454584
S315080068E0454545454545454545454545454545454A
S315080068F0454545454545241E1B2145454527452A09
S315080069002D30FFF701FF29E0FFF71EFF26E0FFF70E
S3150800691099FE23E0FFF7A2FE20E0FFF77DFE1DE0CB
S31508006920FFF774FE1AE0FFF761FE17E0FFF750FE67
S3150800693014E0FFF729FF11E0FFF746FF0EE0FFF727
S31508006940A7FE0BE0FFF76EFF08E0FFF77FFF05E005
S31508006950FFF798FE02E02020FFF730FE0A4B93F877
S315080069604330012B02D11020FFF728FE064BB3F95E
S315080069704410002906DD1846012380F84330033009
S31508006980FFF770FF08BD00BFBC17002008B5074B0E
S31508006990044613B10021AFF30080054B1868836ADB
S315080069A003B19847204600F033F800BF0000000006
S315080069B02073000870B50E4B0E4CE41AA41000257F
S315080069C01E46A54204D056F8253098470135F8E703
S315080069D000F020F8084C094BE41AA41000251E46BE
S315080069E0A54204D056F8253098470135F8E770BD1A
S315080069F048010020480100204C01002048010020E1
S31508006A0002440346934202D003F8011BFAE7704793
S31508006A10FEE70000F8B500BFF8BC08BC9E46704704
S31508006A20F8B500BFF8BC08BC9E4670472F64656D74
S31508006A306F70726F675F6F6C696D65785F73746D81
S31508006A403332703430352E73726563002F626F6F80
S31508006A50746C6F672E7478740000000057696E5561
S31508006A6053422042756C6B20446576696365000065
S31508006A704F70656E424C54205573657200000000D5
S31508006A8030303030303030303035304300000000A0
S31508006A9044656661756C740057696E5553422042A9
S31508006AA0756C6B20496E74657266616365000000DB
S31508006AB02E2E5C2E2E5C2E2E5C2E2E5C536F75723F
S31508006AC063655C41524D434D345F53544D333246F2
S31508006AD0345C63616E2E6300050206020603070333
S31508006AE00803090309040A040B040C040C050D0524
S31508006AF00E050F050F0610061007100800000800FF
S31508006B001000180020002800300038004000480017
S31508006B10500058008000880090009800A000A80047
S31508006B20B000B800C000C800D000D8000080000837
S31508006B30004000000200000000C0000800400000FD
S31508006B400300000000000108000001000400000026
S31508006B50000002080000020005000000000004080A
S31508006B6000000200060000000000060800000200FF
S31508006B7007000000000008080000020008000000E6
S31508006B8000000A08000002000900000000000C08C6
S31508006B90000002000A00000000000E0800000200C3
S31508006BA00B0000002E2E5C2E2E5C2E2E5C2E2E5CEC
S31508006BB0536F757263655C41524D434D345F535450
S31508006BC04D333246345C756172742E6300000000E2
S31508006BD02E2E5C2E2E5C2E2E5C2E2E5C536F75721E
S31508006BE063655C41524D434D345F53544D333246D1
S31508006BF0345C7573622E6300303A00002E2E5C2ECC
S31508006C002E5C2E2E5C2E2E5C536F757263655C6649
S31508006C10696C652E630000004669726D776172655E
S31508006C20207570646174652072657175657374206A
S31508006C3064657465637465640A0D00004F70656E5B
S31508006C40696E67206669726D776172652066696C20
S31508006C506520666F722072656164696E672E2E2ED6
S31508006C60000000004552524F520A0D004F4B0A0DC4
S31508006C70000000005374617274696E672074686559
S31508006C802070726F6772616D6D696E6720736571CA
S31508006C9075656E63650A0D0050617273696E6720CB
S31508006CA06669726D776172652066696C6520746FB6
S31508006CB02064657465637420657261736520626C0F
S31508006CC06F636B732E2E2E0045726173696E672093
S31508006CD0000000002062797465732066726F6D206B
S31508006CE06D656D6F72792061742030780000000040
S31508006CF052656164696E67206C696E652066726F9D
S31508006D006D2066696C652E2E2E4552524F520A0D1D
S31508006D1000000000496E76616C69642063686563EB
S31508006D206B73756D20666F756E642E2E2E455252E6
S31508006D304F520A0D0000000050726F6772616D6D48
S31508006D40696E6720000000002062797465732074FC
S31508006D506F206D656D6F7279206174203078000040
S31508006D6057726974696E672070726F6772616D20F9
S31508006D70636865636B73756D2E2E2E00436C6F7397
S31508006D80696E67206669726D776172652066696CDF
S31508006D90650A0D004669726D7761726520757064C3
S31508006DA0617465207375636365737366756C6C7956
S31508006DB020636F6D706C657465640A0D00000000D1
S31508006DC0222A3A3C3E3F7C7F000000002B2C3B3DAC
S31508006DD05B5D0000809A45418E418F804545454957
S31508006DE049498E8F9092924F994F555559999A9B2A
S31508006DF09C9D9E9F41494F55A5A5A6A7A8A9AAABA4
S31508006E00ACADAEAFB0B1B2B3B4B5B6B7B8B9BABB3C
S31508006E10BCBDBEBFC0C1C2C3C4C5C6C7C8C9CACB2C
S31508006E20CCCDCECFD0D1D2D3D4D5D6D7D8D9DADB1C
S31508006E30DCDDDEDFE0E1E2E3E4E5E6E7E8E9EAEB0C
S31508006E40ECEDEEEFF0F1F2F3F4F5F6F7F8F9FAFBFC
S31508006E50FCFDFEFF01030507090E10121416181C87
S31508006E601E0000007D1D0100632C001E9601A01E59
S31508006E705A01001F0806101F0606201F0806301FA5
S31508006E800806401F0606511F0700591F521F5B1FA1
S31508006E90541F5D1F561F5F1F601F0806701F0E00D8
S31508006EA0BA1FBB1FC81FC91FCA1FCB1FDA1FDB1F8C
S31508006EB0F81FF91FEA1FEB1FFA1FFB1F801F0806A2
S31508006EC0901F0806A01F0806B01F0400B81FB91FA8
S31508006ED0B21FBC1FCC1F0100C31FD01F0206E01F34
S31508006EE00206E51F0100EC1FF21F0100FC1F4E21E0
S31508006EF00100322170211002842101008321D0244F
S31508006F001A05302C2F04602C0201672C0601752CFB
S31508006F100201802C6401002D260841FF1A03000097
S31508006F2061001A03E0001703F8000703FF000100D9
S31508006F3078010001300132010601390110014A01C8
S31508006F402E017901060180014D004302810182016B
S31508006F5082018401840186018701870189018A01EA
S31508006F608B018B018D018E018F0190019101910199
S31508006F7093019401F60196019701980198013D0243
S31508006F809B019C019D0120029F01A001A001A20175
S31508006F90A201A401A401A601A701A701A901AA01AA
S31508006FA0AB01AC01AC01AE01AF01AF01B101B20159
S31508006FB0B301B301B501B501B701B801B801BA010A
S31508006FC0BB01BC01BC01BE01F701C001C101C20180
S31508006FD0C301C401C501C401C701C801C701CA016B
S31508006FE0CB01CA01CD011001DD0101008E01DE01D0
S31508006FF01201F3010300F101F401F401F80128017B
S31508007000220212013A020900652C3B023B023D02AC
S31508007010662C3F0240024102410246020A0153021F
S31508007020400081018601550289018A0158028F01B3
S315080070305A0290015C025D025E025F0293016102E0
S31508007040620294016402650266026702970196016C
S315080070506A02622C6C026D026E029C017002710259
S315080070609D01730274029F01760277027802790203
S315080070707A027B027C02642C7E027F02A6018102D0
S315080070808202A9018402850286028702AE014402B1
S31508007090B101B20145028D028E028F029002910261
S315080070A0B7017B030300FD03FE03FF03AC030400E3
S315080070B08603880389038A03B1031103C203020006
S315080070C0A303A303C4030803CC0303008C038E03A2
S315080070D08F03D8031801F2030A00F903F303F40334
S315080070E0F503F603F703F703F903FA03FA03300483
S315080070F0200350041007600422018A043601C104E3
S315080071000E01CF040100C004D00444016105260421
S3150800711000000000C700FC00E900E200E400E0000F
S31508007120E500E700EA00EB00E800EF00EE00EC00FF
S31508007130C400C500C900E600C600F400F600F20067
S31508007140FB00F900FF00D600DC00A200A300A500A2
S31508007150A7209201E100ED00F300FA00F100D1004A
S31508007160AA00BA00BF001023AC00BD00BC00A100F5
S31508007170AB00BB0091259225932502252425612580
S315080071806225562555256325512557255D255C25F8
S315080071905B251025142534252C251C2500253C2582
S315080071A05E255F255A2554256925662560255025BF
S315080071B06C25672568256425652559255825522592
S315080071C053256B256A2518250C25882584258C25A5
S315080071D090258025B103DF009303C003A303C303EF
S315080071E0B500C403A6039803A903B4031E22C60365
S315080071F0B50329226122B1006522642220232123B6
S31508007200F7004822B0001922B7001A227F20B200E0
S31508007210A025A0004F70656E424C54000020202027
S315080072202020202020202828282828202020202028
S3150800723020202020202020202020202020881010F8
S315080072401010101010101010101010101004040454
S315080072500404040404040410101010101010414112
S315080072604141414101010101010101010101010100
S315080072700101010101010101101010101010424214
S3150800728042424242020202020202020202020202D0
S315080072900202020202020202101010102000000070
S315080072A000000000000000000000000000000000D0
S315080072B000000000000000000000000000000000C0
S315080072C000000000000000000000000000000000B0
S315080072D000000000000000000000000000000000A0
S315080072E00000000000000000000000000000000090
S315080072F00000000000000000000000000000000080
S31508007300000000000000000000000000000000006F
S31508007310000000000000000000000000004300001C
S30D08007320E8000020000000004F
S30D08007328BC8EFF7F0100000086
S31508007330010000000000000001020304010203042A
S31508007340060708091800002061150008AD14000892
S315080073505D140008C51300082D140008A9130008B9
S3150800736091130008D5130008E5130008F513000863
S315080073700D1400083131000819310008B930000829
S315080073800000000000000000A1300008AD30000831
S315080073908D30000800000000000000008130000861
S315080073A009022000010100C0320904000002FF00A2
S315080073B00000070581024000FF070501024000FFA3
S315080073C069310008753100089D31000881310008CF
S315080073D0B9310008D5310008F13100080403090461
S315080073E01201100100000040501DAC6000010102AE
S315080073F0030100000D32000811320008153200089A
S3150800740019320008213200082932000835320008EE
S31508007410040000001C7200080000000000000000C4
S31508007420000000000000000000000000000000004E
S3150800743000000000000000001D73000800000000A6
S31508007440000000000000000000000000000000002E
S31508007450000000000000000000000000000000001E
S31508007460000000000000000000000000000000000E
S315080074700000000000000000AD01000889010008B6
S70508000000F2
